LX51 LINKER/LOCATER V4.66.97.0                                                          07/19/2022  10:30:28  PAGE 1


LX51 LINKER/LOCATER V4.66.97.0, INVOKED BY:
C:\KEIL_V5\C51\BIN\LX51.EXE .\Out_Files\STARTUP.obj, .\Out_Files\system_um800y.obj, .\Out_Files\common.obj, .\Out_Files\
>> uart0.obj, .\Out_Files\lvd.obj, .\Out_Files\app.obj, .\Out_Files\main.obj TO .\Out_Files\um800y PRINT (.\Out_Files\um
>> 800y.map) REMOVEUNUSED CLASSES (XDATA (X:0X0-X:0X7FF), HDATA (X:0X0-X:0X7FF), ECODE (C:0X0-C:0XFFFF), HCONST (C:0X0-C
>> :0XFFFF))


CPU MODE:     8051 MODE
MEMORY MODEL: LARGE


INPUT MODULES INCLUDED:
  .\Out_Files\STARTUP.obj (?C_STARTUP)
         COMMENT TYPE 1: A51 / ASM51 Assembler
  .\Out_Files\system_um800y.obj (SYSTEM_UM800Y)
         COMMENT TYPE 0: C51 V9.60.0.0
  .\Out_Files\common.obj (COMMON)
         COMMENT TYPE 0: C51 V9.60.0.0
  .\Out_Files\uart0.obj (UART0)
         COMMENT TYPE 0: C51 V9.60.0.0
  .\Out_Files\lvd.obj (LVD)
         COMMENT TYPE 0: C51 V9.60.0.0
  .\Out_Files\app.obj (APP)
         COMMENT TYPE 0: C51 V9.60.0.0
  .\Out_Files\main.obj (MAIN)
         COMMENT TYPE 0: C51 V9.60.0.0
  C:\KEIL_V5\C51\LIB\C51L.LIB (?C_INIT)
         COMMENT TYPE 1: A51 / ASM51 Assembler
  C:\KEIL_V5\C51\LIB\C51L.LIB (?C?CLDPTR)
         COMMENT TYPE 1: A51 / ASM51 Assembler
  C:\KEIL_V5\C51\LIB\C51L.LIB (?C?CLDOPTR)
         COMMENT TYPE 1: A51 / ASM51 Assembler
  C:\KEIL_V5\C51\LIB\C51L.LIB (?C?ILDIX)
         COMMENT TYPE 1: A51 / ASM51 Assembler
  C:\KEIL_V5\C51\LIB\C51L.LIB (?C?LADD)
         COMMENT TYPE 1: A51 / ASM51 Assembler
  C:\KEIL_V5\C51\LIB\C51L.LIB (?C?LMUL)
         COMMENT TYPE 1: A51 / ASM51 Assembler
  C:\KEIL_V5\C51\LIB\C51L.LIB (?C?ULDIV)
         COMMENT TYPE 1: A51 / ASM51 Assembler
  C:\KEIL_V5\C51\LIB\C51L.LIB (?C?LOR)
         COMMENT TYPE 1: A51 / ASM51 Assembler
  C:\KEIL_V5\C51\LIB\C51L.LIB (?C?ULCMP)
         COMMENT TYPE 1: A51 / ASM51 Assembler
  C:\KEIL_V5\C51\LIB\C51L.LIB (?C?ULSHR)
         COMMENT TYPE 1: A51 / ASM51 Assembler
  C:\KEIL_V5\C51\LIB\C51L.LIB (?C?LSHL)
         COMMENT TYPE 1: A51 / ASM51 Assembler
  C:\KEIL_V5\C51\LIB\C51L.LIB (?C?LLDOPTR)
         COMMENT TYPE 1: A51 / ASM51 Assembler
  C:\KEIL_V5\C51\LIB\C51L.LIB (?C?LLDXDATA)
         COMMENT TYPE 1: A51 / ASM51 Assembler
  C:\KEIL_V5\C51\LIB\C51L.LIB (?C?LLDXDATA0)
         COMMENT TYPE 1: A51 / ASM51 Assembler
  C:\KEIL_V5\C51\LIB\C51L.LIB (?C?LLDIXDATA)
         COMMENT TYPE 1: A51 / ASM51 Assembler
  C:\KEIL_V5\C51\LIB\C51L.LIB (?C?LSTXDATA)
         COMMENT TYPE 1: A51 / ASM51 Assembler
  C:\KEIL_V5\C51\LIB\C51L.LIB (?C?LSTKXDATA)
         COMMENT TYPE 1: A51 / ASM51 Assembler
  C:\KEIL_V5\C51\LIB\C51L.LIB (?C?PLDXDATA)
         COMMENT TYPE 1: A51 / ASM51 Assembler
  C:\KEIL_V5\C51\LIB\C51L.LIB (?C?PLDIXDATA)
         COMMENT TYPE 1: A51 / ASM51 Assembler
  C:\KEIL_V5\C51\LIB\C51L.LIB (?C?PSTXDATA)
         COMMENT TYPE 1: A51 / ASM51 Assembler
LX51 LINKER/LOCATER V4.66.97.0                                                        07/19/2022  10:30:28  PAGE 2


  C:\KEIL_V5\C51\LIB\C51L.LIB (?C?LCASE)
         COMMENT TYPE 1: A51 / ASM51 Assembler
  C:\KEIL_V5\C51\LIB\C51L.LIB (?C?ICALL)
         COMMENT TYPE 1: A51 / ASM51 Assembler
  C:\KEIL_V5\C51\LIB\C51L.LIB (PRINTF)
         COMMENT TYPE 1: A51 / ASM51 Assembler
  C:\KEIL_V5\C51\LIB\C51L.LIB (?C?CSTPTR)
         COMMENT TYPE 1: A51 / ASM51 Assembler
  C:\KEIL_V5\C51\LIB\C51L.LIB (?C?LLDIDATA)
         COMMENT TYPE 1: A51 / ASM51 Assembler
  C:\KEIL_V5\C51\LIB\C51L.LIB (?C?LLDPDATA)
         COMMENT TYPE 1: A51 / ASM51 Assembler
  C:\KEIL_V5\C51\LIB\C51L.LIB (?C?LLDCODE)
         COMMENT TYPE 1: A51 / ASM51 Assembler
  C:\KEIL_V5\C51\LIB\C51L.LIB (?C?CCASE)
         COMMENT TYPE 1: A51 / ASM51 Assembler


ACTIVE MEMORY CLASSES OF MODULE:  .\Out_Files\um800y (?C_STARTUP)

BASE        START       END         USED      MEMORY CLASS
==========================================================
X:000000H   X:000000H   X:0007FFH   00007AH   XDATA
X:000000H   X:000000H   X:0007FFH             HDATA
C:000000H   C:000000H   C:00FFFFH             ECODE
C:000000H   C:000000H   C:00FFFFH             HCONST
C:000000H   C:000000H   C:00FFFFH   000A7EH   CODE
I:000000H   I:000000H   I:0000FFH   000001H   IDATA
C:000000H   C:000000H   C:00FFFFH   000033H   CONST
I:000000H   I:000000H   I:00007FH   00000DH   DATA
I:000020H.0 I:000020H.0 I:00002FH.7 000001H.1 BIT


MEMORY MAP OF MODULE:  .\Out_Files\um800y (?C_STARTUP)


START     STOP      LENGTH    ALIGN  RELOC    MEMORY CLASS   SEGMENT NAME
=========================================================================

* * * * * * * * * * *   D A T A   M E M O R Y   * * * * * * * * * * * * *
000000H   000007H   000008H   ---    AT..     DATA           "REG BANK 0"
000008H   00000CH   000005H   BYTE   UNIT     DATA           _DATA_GROUP_
00000DH.0 00001FH.7 000013H.0 ---    ---      **GAP**
000020H.0 000021H.0 000001H.1 BIT    UNIT     BIT            _BIT_GROUP_
000021H.1 000021H   000000H.7 ---    ---      **GAP**
000022H   000022H   000001H   BYTE   UNIT     IDATA          ?STACK

* * * * * * * * * * *   C O D E   M E M O R Y   * * * * * * * * * * * * *
000000H   000002H   000003H   ---    OFFS..   CODE           ?CO??C_STARTUP?0
000003H   000020H   00001EH   BYTE   UNIT     CODE           ?PR?EFC_IRQHANDLER?LVD
000021H   000022H   000002H   ---    ---      **GAP**
000023H   000025H   000003H   BYTE   OFFS..   CODE           ?UART0?00023
000026H   00004CH   000027H   BYTE   UNIT     CODE           ?C_INITSEG
00004DH   000057H   00000BH   BYTE   UNIT     CODE           ?PR?SYSTEM_INIT?SYSTEM_UM800Y
000058H   00005AH   000003H   BYTE   UNIT     CODE           ?PR?UART0_RECV_BYTE?UART0
00005BH   00005DH   000003H   BYTE   OFFS..   CODE           ?LVD?0005B
00005EH   0003C2H   000365H   BYTE   UNIT     CODE           ?PR?PRINTF?PRINTF
0003C3H   00070FH   00034DH   BYTE   UNIT     CODE           ?C?LIB_CODE
000710H   00083DH   00012EH   BYTE   UNIT     CODE           ?PR?_CLOCK_INIT?SYSTEM_UM800Y
00083EH   0008C9H   00008CH   BYTE   UNIT     CODE           ?C_C51STARTUP
0008CAH   000940H   000077H   BYTE   UNIT     CODE           ?PR?_UART0_SET_BAUD_RATE?UART0
000941H   00098AH   00004AH   BYTE   UNIT     CODE           ?PR?UART0_IRQHANDLER?UART0
00098BH   0009C3H   000039H   BYTE   UNIT     CODE           ?PR?LVD_TEST?APP
0009C4H   0009FAH   000037H   BYTE   UNIT     CODE           ?PR?_UART0_INIT?UART0
0009FBH   000A1CH   000022H   BYTE   UNIT     CODE           ?PR?UART0_REC_PRO?APP
LX51 LINKER/LOCATER V4.66.97.0                                                        07/19/2022  10:30:28  PAGE 3


000A1DH   000A35H   000019H   BYTE   UNIT     CODE           ?PR?UART_INIT?APP
000A36H   000A4BH   000016H   BYTE   UNIT     CODE           ?PR?_UART0_SEND_BYTE?UART0
000A4CH   000A5DH   000012H   BYTE   UNIT     CODE           ?PR?_UART0_IRQ_INIT?UART0
000A5EH   000A6FH   000012H   BYTE   UNIT     CODE           ?PR?LVD_INIT?LVD
000A70H   000A7AH   00000BH   BYTE   UNIT     CODE           ?PR?MAIN?MAIN
000A7BH   000A7FH   000005H   BYTE   UNIT     CODE           ?PR?_PUTCHAR?UART0
000A80H   000AB2H   000033H   BYTE   UNIT     CONST          ?CO?APP

* * * * * * * * * * *  X D A T A   M E M O R Y  * * * * * * * * * * * * *
000000H   000044H   000045H   BYTE   UNIT     XDATA          ?XD?APP
000045H   00006CH   000028H   BYTE   UNIT     XDATA          _XDATA_GROUP_
00006DH   000074H   000008H   BYTE   UNIT     XDATA          ?XD?SYSTEM_UM800Y
000075H   000078H   000004H   BYTE   UNIT     XDATA          ?XD?UART0
000079H   000079H   000001H   BYTE   UNIT     XDATA          ?XD?LVD

* * * * * * * * *   R E M O V E D     S E G M E N T S   * * * * * * * *
   *DEL*:           000047H   BYTE   UNIT     CODE           ?PR?_DELAY1MS?COMMON
   *DEL*:           000008H   BYTE   UNIT     XDATA          ?XD?_DELAY1MS?COMMON
   *DEL*:           000015H   BYTE   UNIT     CODE           ?PR?_DELAY?COMMON
   *DEL*:           000004H   BYTE   UNIT     XDATA          ?XD?_DELAY?COMMON
   *DEL*:           00006CH   BYTE   UNIT     CODE           ?PR?_PRINTF_BUFF_BYTE?COMMON
   *DEL*:           00000BH   BYTE   UNIT     XDATA          ?XD?_PRINTF_BUFF_BYTE?COMMON
   *DEL*:           000077H   BYTE   UNIT     CODE           ?PR?_PRINTF_BUFF_WORD?COMMON
   *DEL*:           00000BH   BYTE   UNIT     XDATA          ?XD?_PRINTF_BUFF_WORD?COMMON
   *DEL*:           000010H   BYTE   UNIT     CONST          ?CO?COMMON
   *DEL*:           00002EH   BYTE   UNIT     CODE           ?PR?_UART0_SEND_BYTES?UART0
   *DEL*:           000007H   BYTE   UNIT     XDATA          ?XD?_UART0_SEND_BYTES?UART0



OVERLAY MAP OF MODULE:   .\Out_Files\um800y (?C_STARTUP)


FUNCTION/MODULE                  BIT_GROUP   DATA_GROUP   XDATA_GROUP
--> CALLED FUNCTION/MODULE      START  STOP  START  STOP  START  STOP
=====================================================================
?C_C51STARTUP                   ----- -----  ----- -----  ----- -----
  +--> MAIN/MAIN
  +--> ?C_INITSEG

MAIN/MAIN                       ----- -----  ----- -----  ----- -----
  +--> SYSTEM_INIT/SYSTEM_UM800Y
  +--> UART_INIT/APP
  +--> LVD_TEST/APP

SYSTEM_INIT/SYSTEM_UM800Y       ----- -----  ----- -----  ----- -----
  +--> _CLOCK_INIT/SYSTEM_UM800Y

_CLOCK_INIT/SYSTEM_UM800Y       ----- -----  ----- -----  0045H 004CH

UART_INIT/APP                   ----- -----  ----- -----  ----- -----
  +--> _UART0_INIT/UART0
  +--> UART0_REC_PRO/APP
  +--> _UART0_IRQ_INIT/UART0

_UART0_INIT/UART0               ----- -----  ----- -----  0045H 0048H
  +--> _UART0_SET_BAUD_RATE/UART0

_UART0_SET_BAUD_RATE/UART0      ----- -----  ----- -----  0049H 0054H

UART0_REC_PRO/APP               ----- -----  ----- -----  ----- -----
  +--> UART0_RECV_BYTE/UART0

UART0_RECV_BYTE/UART0           ----- -----  ----- -----  ----- -----

LX51 LINKER/LOCATER V4.66.97.0                                                        07/19/2022  10:30:28  PAGE 4


_UART0_IRQ_INIT/UART0           ----- -----  ----- -----  ----- -----

LVD_TEST/APP                    ----- -----  ----- -----  ----- -----
  +--> PRINTF/PRINTF
  +--> LVD_INIT/LVD

PRINTF/PRINTF                   20H.0 21H.0  0008H 000CH  0045H 006CH
  +--> _PUTCHAR/UART0

_PUTCHAR/UART0                  ----- -----  ----- -----  ----- -----
  +--> _UART0_SEND_BYTE/UART0

_UART0_SEND_BYTE/UART0          ----- -----  ----- -----  ----- -----

LVD_INIT/LVD                    ----- -----  ----- -----  ----- -----

?C_INITSEG                      ----- -----  ----- -----  ----- -----

*** NEW ROOT ******************

UART0_IRQHANDLER/UART0          ----- -----  ----- -----  ----- -----

*** NEW ROOT ******************

EFC_IRQHANDLER/LVD              ----- -----  ----- -----  ----- -----



PUBLIC SYMBOLS OF MODULE:  .\Out_Files\um800y (?C_STARTUP)


      VALUE       CLASS    TYPE      PUBLIC SYMBOL NAME
      =================================================
      02000045H   XDATA    ---       ?_PRINTF517?BYTE
      02000045H   XDATA    ---       ?_PRINTF?BYTE
      02000045H   XDATA    ---       ?_SPRINTF517?BYTE
      02000045H   XDATA    ---       ?_SPRINTF?BYTE
      010006EAH   CODE     ---       ?C?CCASE
      010003DCH   CODE     ---       ?C?CLDOPTR
      010003C3H   CODE     ---       ?C?CLDPTR
      00000000H   NUMBER   ---       ?C?CODESEG
      010006B0H   CODE     ---       ?C?CSTPTR
      010006AAH   CODE     ---       ?C?ICALL
      010006AEH   CODE     ---       ?C?ICALL2
      01000409H   CODE     ---       ?C?ILDIX
      0100041FH   CODE     ---       ?C?LADD
      01000670H   CODE     ---       ?C?LCASE
      010006DAH   CODE     ---       ?C?LLDCODE
      010006C2H   CODE     ---       ?C?LLDIDATA
      010005DEH   CODE     ---       ?C?LLDIXDATA
      010005D5H   CODE     ---       ?C?LLDIXDATA1
      010005D7H   CODE     ---       ?C?LLDIXDATA8
      0100058DH   CODE     ---       ?C?LLDOPTR
      010006CEH   CODE     ---       ?C?LLDPDATA
      010005BDH   CODE     ---       ?C?LLDXDATA
      010005C9H   CODE     ---       ?C?LLDXDATA0
      0100042CH   CODE     ---       ?C?LMUL
      01000549H   CODE     ---       ?C?LOR
      0100057AH   CODE     ---       ?C?LSHL
      01000616H   CODE     ---       ?C?LSTKXDATA
      0100060AH   CODE     ---       ?C?LSTXDATA
      01000650H   CODE     ---       ?C?PLDIXDATA
      01000647H   CODE     ---       ?C?PLDXDATA
      01000667H   CODE     ---       ?C?PSTXDATA
      01000556H   CODE     ---       ?C?ULCMP
LX51 LINKER/LOCATER V4.66.97.0                                                        07/19/2022  10:30:28  PAGE 5


      010004B7H   CODE     ---       ?C?ULDIV
      01000567H   CODE     ---       ?C?ULSHR
      00000000H   NUMBER   ---       ?C?XDATASEG
      01000885H   CODE     ---       ?C_START
      01000000H   CODE     ---       ?C_STARTUP
      01000710H   CODE     ---       _clock_init
*DEL*:00000000H   CODE     ---       _delay
*DEL*:00000000H   CODE     ---       _delay1ms
      010000C9H   CODE     ---       _PRINTF
      010000C9H   CODE     ---       _PRINTF517
*DEL*:00000000H   CODE     ---       _printf_buff_byte
*DEL*:00000000H   CODE     ---       _printf_buff_word
      01000A7BH   CODE     ---       _putchar
      010000C3H   CODE     ---       _SPRINTF
      010000C3H   CODE     ---       _SPRINTF517
      010009C4H   CODE     ---       _uart0_init
      01000A4CH   CODE     ---       _uart0_irq_init
      01000A36H   CODE     ---       _uart0_send_byte
*DEL*:00000000H   CODE     ---       _uart0_send_bytes
*SFR* 000000D0H.6 DATA     BIT       AC
*SFR* 000000E0H   DATA     BYTE      ACC
*SFR* 000000E0H.0 DATA     BIT       ACC0
*SFR* 000000E0H.1 DATA     BIT       ACC1
*SFR* 000000E0H.2 DATA     BIT       ACC2
*SFR* 000000E0H.3 DATA     BIT       ACC3
*SFR* 000000E0H.4 DATA     BIT       ACC4
*SFR* 000000E0H.5 DATA     BIT       ACC5
*SFR* 000000E0H.6 DATA     BIT       ACC6
*SFR* 000000E0H.7 DATA     BIT       ACC7
*SFR* 000000FEH   DATA     BYTE      ADCCDR0
*SFR* 000000FFH   DATA     BYTE      ADCCDR1
*SFR* 000000F6H   DATA     BYTE      ADCCSTAT
*SFR* 000000B6H   DATA     WORD      ADCDR
*SFR* 000000B6H   DATA     BYTE      ADCDR0
*SFR* 000000B7H   DATA     BYTE      ADCDR1
*SFR* 000000ACH   DATA     BYTE      ADCGCR0
*SFR* 000000ADH   DATA     BYTE      ADCGCR1
*SFR* 000000B4H   DATA     BYTE      ADCGCR2
*SFR* 000000B5H   DATA     BYTE      ADCGCR3
*SFR* 000000F5H   DATA     BYTE      ADCHL
*SFR* 00000093H   DATA     BYTE      ADCIER
*SFR* 000000F7H   DATA     BYTE      ADCSPW
*SFR* 000000FDH   DATA     BYTE      ADCVREF
*SFR* 000000F0H   DATA     BYTE      B
*SFR* 000000F0H.0 DATA     BIT       B0
*SFR* 000000F0H.1 DATA     BIT       B1
*SFR* 000000F0H.2 DATA     BIT       B2
*SFR* 000000F0H.3 DATA     BIT       B3
*SFR* 000000F0H.4 DATA     BIT       B4
*SFR* 000000F0H.5 DATA     BIT       B5
*SFR* 000000F0H.6 DATA     BIT       B6
*SFR* 000000F0H.7 DATA     BIT       B7
*SFR* 00000086H   DATA     BYTE      BEEPCTR
*SFR* 000000F8H   DATA     BYTE      CLKCON
*SFR* 000000B1H   DATA     BYTE      CLKST
*SFR* 000000D0H.7 DATA     BIT       CY
*SFR* 00000083H   DATA     BYTE      DPH
*SFR* 00000085H   DATA     BYTE      DPH1
*SFR* 00000082H   DATA     BYTE      DPL
*SFR* 00000084H   DATA     BYTE      DPL1
*SFR* 00000092H   DATA     BYTE      DPS
*SFR* 000000A8H.7 DATA     BIT       EA
*SFR* 000000A8H.6 DATA     BIT       EADC
      01000003H   CODE     ---       EFC_IRQHandler
*SFR* 000000B8H.3 DATA     BIT       EFCINTEN
LX51 LINKER/LOCATER V4.66.97.0                                                        07/19/2022  10:30:28  PAGE 6


*SFR* 000000A8H.5 DATA     BIT       EPWM
*SFR* 000000D8H.3 DATA     BIT       ERSTF
*SFR* 000000A8H.4 DATA     BIT       ES0
*SFR* 000000A8H.2 DATA     BIT       ES1
*SFR* 000000B2H   DATA     BYTE      ESTCR
*SFR* 000000A8H.1 DATA     BIT       ET0
*SFR* 000000A8H.3 DATA     BIT       ET1
*SFR* 0000009EH   DATA     BYTE      EUARTEN
*SFR* 000000A8H.0 DATA     BIT       EX0
*SFR* 000000D0H.5 DATA     BIT       F0
*SFR* 000000D0H.1 DATA     BIT       F1
*SFR* 000000B8H.0 DATA     BIT       GTIM0INTEN
*SFR* 000000B8H.2 DATA     BIT       GTIM1INTEN
*SFR* 000000B8H.6 DATA     BIT       GTIM2INTEN
*SFR* 000000B8H.5 DATA     BIT       I2CINTEN
*SFR* 000000A8H   DATA     BYTE      IEN0
*SFR* 000000B8H   DATA     BYTE      IEN1
*SFR* 0000009AH   DATA     BYTE      IEN2
*SFR* 000000A9H   DATA     BYTE      IP0
*SFR* 000000B9H   DATA     BYTE      IP1
*SFR* 000000BDH   DATA     BYTE      LDOTRIMH
*SFR* 00000091H   DATA     BYTE      LDOTRIML
*SFR* 000000B8H.4 DATA     BIT       LPTIMINTEN
      02000079H   XDATA    BYTE      lvd_flag
      01000A5EH   CODE     ---       lvd_init
      0100098BH   CODE     ---       lvd_test
*SFR* 000000DDH   DATA     BYTE      LVDCON
*SFR* 000000D8H.5 DATA     BIT       LVRF
      01000A70H   CODE     ---       main
*SFR* 000000D1H   DATA     WORD      OADR
*SFR* 000000D2H   DATA     BYTE      OADRH
*SFR* 000000D1H   DATA     BYTE      OADRL
*SFR* 000000D4H   DATA     BYTE      OCTRL
*SFR* 000000D3H   DATA     BYTE      ODATA
*SFR* 000000A2H   DATA     BYTE      OINTEN
*SFR* 000000A3H   DATA     BYTE      OINTUS
*SFR* 000000A7H   DATA     BYTE      OPSET
*SFR* 000000A5H   DATA     BYTE      OSEC
*SFR* 000000A6H   DATA     BYTE      OSTATUS
*SFR* 000000A1H   DATA     BYTE      OUS
*SFR* 000000D0H.0 DATA     BIT       P
*SFR* 00000080H   DATA     BYTE      P0
*SFR* 00000080H.0 DATA     BIT       P00
*SFR* 00000080H.1 DATA     BIT       P01
*SFR* 00000080H.2 DATA     BIT       P02
*SFR* 00000080H.3 DATA     BIT       P03
*SFR* 00000080H.4 DATA     BIT       P04
*SFR* 00000080H.5 DATA     BIT       P05
*SFR* 000000ABH   DATA     BYTE      P0AH
*SFR* 000000A4H   DATA     BYTE      P0AL
*SFR* 000000D7H   DATA     BYTE      P0CS
*SFR* 00000097H   DATA     BYTE      P0DR
*SFR* 000000E9H   DATA     BYTE      P0IEN
*SFR* 000000E1H   DATA     BYTE      P0IRQ
*SFR* 000000D6H   DATA     BYTE      P0OD
*SFR* 000000F9H   DATA     BYTE      P0OEN
*SFR* 000000D5H   DATA     BYTE      P0PD
*SFR* 000000F1H   DATA     BYTE      P0PU
*SFR* 00000090H   DATA     BYTE      P1
*SFR* 00000090H.0 DATA     BIT       P10
*SFR* 00000090H.1 DATA     BIT       P11
*SFR* 00000090H.2 DATA     BIT       P12
*SFR* 00000090H.3 DATA     BIT       P13
*SFR* 00000090H.4 DATA     BIT       P14
*SFR* 00000090H.5 DATA     BIT       P15
LX51 LINKER/LOCATER V4.66.97.0                                                        07/19/2022  10:30:28  PAGE 7


*SFR* 000000B0H   DATA     BYTE      P1AH
*SFR* 000000AEH   DATA     BYTE      P1AL
*SFR* 000000DCH   DATA     BYTE      P1CS
*SFR* 000000E5H   DATA     BYTE      P1DR
*SFR* 000000EAH   DATA     BYTE      P1IEN
*SFR* 000000E2H   DATA     BYTE      P1IRQ
*SFR* 000000DBH   DATA     BYTE      P1OD
*SFR* 000000FAH   DATA     BYTE      P1OEN
*SFR* 000000DAH   DATA     BYTE      P1PD
*SFR* 000000F2H   DATA     BYTE      P1PU
*SFR* 000000A0H   DATA     BYTE      P2
*SFR* 000000A0H.0 DATA     BIT       P20
*SFR* 000000A0H.2 DATA     BIT       P22
*SFR* 000000A0H.3 DATA     BIT       P23
*SFR* 000000A0H.5 DATA     BIT       P25
*SFR* 000000A0H.6 DATA     BIT       P26
*SFR* 000000A0H.7 DATA     BIT       P27
*SFR* 000000E8H   DATA     BYTE      P2AH
*SFR* 000000C0H   DATA     BYTE      P2AL
*SFR* 000000F4H   DATA     BYTE      P2CS
*SFR* 000000FCH   DATA     BYTE      P2DR
*SFR* 000000EBH   DATA     BYTE      P2IEN
*SFR* 000000E3H   DATA     BYTE      P2IRQ
*SFR* 000000ECH   DATA     BYTE      P2OD
*SFR* 000000FBH   DATA     BYTE      P2OEN
*SFR* 000000E4H   DATA     BYTE      P2PD
*SFR* 000000F3H   DATA     BYTE      P2PU
*SFR* 000000DEH   DATA     BYTE      PCLK0
*SFR* 000000DFH   DATA     BYTE      PCLK1
*SFR* 00000087H   DATA     BYTE      PCON
*SFR* 0000008EH   DATA     BYTE      PDSEL
*SFR* 0000008FH   DATA     BYTE      POREN
*SFR* 000000D8H.4 DATA     BIT       PORF
*SFR* 000000E6H   DATA     BYTE      PRESET0
*SFR* 000000E7H   DATA     BYTE      PRESET1
*SFR* 000000D0H   DATA     BYTE      PSW
*SFR* 000000C8H   DATA     BYTE      PWM0CON
*SFR* 000000C4H   DATA     BYTE      PWM0DH
*SFR* 000000C3H   DATA     BYTE      PWM0DL
*SFR* 000000C8H.7 DATA     BIT       PWM0EN
*SFR* 000000C8H.2 DATA     BIT       PWM0IE
*SFR* 000000C8H.1 DATA     BIT       PWM0IF
*SFR* 000000CCH   DATA     BYTE      PWM0PH
*SFR* 000000CBH   DATA     BYTE      PWM0PL
*SFR* 000000C8H.6 DATA     BIT       PWM0S
*SFR* 000000C8H.0 DATA     BIT       PWM0SS
*SFR* 000000C9H   DATA     BYTE      PWM1CON
*SFR* 000000C6H   DATA     BYTE      PWM1DH
*SFR* 000000C5H   DATA     BYTE      PWM1DL
*SFR* 000000CEH   DATA     BYTE      PWM1PH
*SFR* 000000CDH   DATA     BYTE      PWM1PL
*SFR* 000000CAH   DATA     BYTE      PWM2CON
*SFR* 000000C7H   DATA     BYTE      PWM2DH
*SFR* 000000CFH   DATA     BYTE      PWM2DL
*SFR* 000000C2H   DATA     BYTE      PWM2PH
*SFR* 000000C1H   DATA     BYTE      PWM2PL
*SFR* 00000098H.2 DATA     BIT       RB80
*SFR* 000000F8H.2 DATA     BIT       RC16MEN
*SFR* 000000F8H.5 DATA     BIT       RC16MF
*SFR* 000000F8H.3 DATA     BIT       RC32KEN
*SFR* 000000F8H.6 DATA     BIT       RC32KF
      0200006DH   XDATA    DWORD     rch24m
*SFR* 000000EEH   DATA     BYTE      RCHDIV
*SFR* 000000BEH   DATA     BYTE      RCHTRIMH
*SFR* 000000BFH   DATA     BYTE      RCHTRIML
LX51 LINKER/LOCATER V4.66.97.0                                                        07/19/2022  10:30:28  PAGE 8


*SFR* 0000009FH   DATA     BYTE      RCLTRIMH
*SFR* 000000BCH   DATA     BYTE      RCLTRIML
*SFR* 000000AFH   DATA     BYTE      REMAP
*SFR* 00000098H.4 DATA     BIT       REN0
*SFR* 00000098H.0 DATA     BIT       RI0
*SFR* 000000D0H.3 DATA     BIT       RS0
*SFR* 000000D0H.4 DATA     BIT       RS1
*SFR* 000000D8H   DATA     BYTE      RSTSTAT
      02000041H   XDATA    WORD      rx_count
      02000040H   XDATA    BYTE      rx_flag
*SFR* 00000099H   DATA     BYTE      S0BUF
*SFR* 00000098H   DATA     BYTE      S0CON
*SFR* 000000BAH   DATA     BYTE      S0RELH
*SFR* 000000AAH   DATA     BYTE      S0RELL
*SFR* 0000009CH   DATA     BYTE      S1BUF
*SFR* 0000009BH   DATA     BYTE      S1CON
*SFR* 000000BBH   DATA     BYTE      S1RELH
*SFR* 0000009DH   DATA     BYTE      S1RELL
*SFR* 00000098H.7 DATA     BIT       SM0
*SFR* 00000098H.6 DATA     BIT       SM1
*SFR* 00000098H.5 DATA     BIT       SM20
*SFR* 00000081H   DATA     BYTE      SP
*SFR* 000000B8H.1 DATA     BIT       SPIINTEN
*SFR* 000000D9H   DATA     BYTE      SYSDIV
*SFR* 000000F8H.0 DATA     BIT       SYSSEL
      02000071H   XDATA    DWORD     system_core_clock
      0100004DH   CODE     ---       system_init
*SFR* 00000098H.3 DATA     BIT       TB80
*SFR* 00000098H.1 DATA     BIT       TI0
      02000043H   XDATA    WORD      tx_count
      02000075H   XDATA    BYTE      tx_flag
      02000076H   XDATA    ---       uart0_func
      01000941H   CODE     ---       UART0_IRQHandler
      010009FBH   CODE     ---       uart0_rec_pro
      01000058H   CODE     ---       uart0_recv_byte
      02000000H   XDATA    ---       uart0_rx_buf
      02000020H   XDATA    ---       uart0_tx_buf
*SFR* 000000B8H.7 DATA     BIT       UART2INTEN
      01000A1DH   CODE     ---       uart_init
*SFR* 000000D8H.6 DATA     BIT       WDEN
*SFR* 000000D8H.7 DATA     BIT       WDOF
*SFR* 000000D8H.0 DATA     BIT       WDT0
*SFR* 000000D8H.1 DATA     BIT       WDT1
*SFR* 000000D8H.2 DATA     BIT       WDT2
*SFR* 000000F8H.1 DATA     BIT       XCLKEN
*SFR* 000000F8H.4 DATA     BIT       XCLKF
*SFR* 000000B3H   DATA     BYTE      XTHCTR



SYMBOL TABLE OF MODULE:  .\Out_Files\um800y (?C_STARTUP)

      VALUE       REP       CLASS    TYPE      SYMBOL NAME
      ====================================================
      ---         MODULE    ---      ---       ?C_STARTUP
      01000000H   PUBLIC    CODE     ---       ?C_STARTUP
      000000E0H   SYMBOL    DATA     ---       ACC
      000000F0H   SYMBOL    DATA     ---       B
      00000083H   SYMBOL    DATA     ---       DPH
      00000082H   SYMBOL    DATA     ---       DPL
      00000000H   SYMBOL    NUMBER   ---       IBPSTACK
      00000100H   SYMBOL    NUMBER   ---       IBPSTACKTOP
      00000080H   SYMBOL    NUMBER   ---       IDATALEN
      01000841H   SYMBOL    CODE     ---       IDATALOOP
      00000000H   SYMBOL    NUMBER   ---       PBPSTACK
LX51 LINKER/LOCATER V4.66.97.0                                                        07/19/2022  10:30:28  PAGE 9


      00000100H   SYMBOL    NUMBER   ---       PBPSTACKTOP
      00000000H   SYMBOL    NUMBER   ---       PDATALEN
      00000000H   SYMBOL    NUMBER   ---       PDATASTART
      00000000H   SYMBOL    NUMBER   ---       PPAGE
      00000000H   SYMBOL    NUMBER   ---       PPAGEENABLE
      000000A0H   SYMBOL    DATA     ---       PPAGE_SFR
      00000081H   SYMBOL    DATA     ---       SP
      0100083EH   SYMBOL    CODE     ---       STARTUP1
      00000000H   SYMBOL    NUMBER   ---       XBPSTACK
      00000000H   SYMBOL    NUMBER   ---       XBPSTACKTOP
      00000000H   SYMBOL    NUMBER   ---       XDATALEN
      00000000H   SYMBOL    NUMBER   ---       XDATASTART
      01000000H   LINE      CODE     ---       #126
      0100083EH   LINE      CODE     ---       #134
      01000840H   LINE      CODE     ---       #135
      01000841H   LINE      CODE     ---       #136
      01000842H   LINE      CODE     ---       #137
      01000844H   LINE      CODE     ---       #191
      01000847H   LINE      CODE     ---       #205

      ---         MODULE    ---      ---       SYSTEM_UM800Y
      02000071H   PUBLIC    XDATA    DWORD     system_core_clock
      0200006DH   PUBLIC    XDATA    DWORD     rch24m
      0100004DH   PUBLIC    CODE     ---       system_init
      01000710H   PUBLIC    CODE     ---       _clock_init
      00000098H.3 SFRSYM    DATA     BIT       TB80
      000000E0H.7 SFRSYM    DATA     BIT       ACC7
      00000080H   SFRSYM    DATA     BYTE      P0
      00000090H   SFRSYM    DATA     BYTE      P1
      000000A0H   SFRSYM    DATA     BYTE      P2
      00000098H.5 SFRSYM    DATA     BIT       SM20
      000000B2H   SFRSYM    DATA     BYTE      ESTCR
      000000B1H   SFRSYM    DATA     BYTE      CLKST
      000000D0H.6 SFRSYM    DATA     BIT       AC
      000000D8H.3 SFRSYM    DATA     BIT       ERSTF
      000000E6H   SFRSYM    DATA     BYTE      PRESET0
      000000D4H   SFRSYM    DATA     BYTE      OCTRL
      000000A8H.7 SFRSYM    DATA     BIT       EA
      0000008FH   SFRSYM    DATA     BYTE      POREN
      000000C8H   SFRSYM    DATA     BYTE      PWM0CON
      000000E7H   SFRSYM    DATA     BYTE      PRESET1
      000000C9H   SFRSYM    DATA     BYTE      PWM1CON
      00000086H   SFRSYM    DATA     BYTE      BEEPCTR
      000000CAH   SFRSYM    DATA     BYTE      PWM2CON
      000000B8H.4 SFRSYM    DATA     BIT       LPTIMINTEN
      000000ABH   SFRSYM    DATA     BYTE      P0AH
      000000B0H   SFRSYM    DATA     BYTE      P1AH
      000000E8H   SFRSYM    DATA     BYTE      P2AH
      000000F8H.6 SFRSYM    DATA     BIT       RC32KF
      000000A8H   SFRSYM    DATA     BYTE      IEN0
      000000A7H   SFRSYM    DATA     BYTE      OPSET
      000000A4H   SFRSYM    DATA     BYTE      P0AL
      000000B8H   SFRSYM    DATA     BYTE      IEN1
      000000A8H.6 SFRSYM    DATA     BIT       EADC
      00000085H   SFRSYM    DATA     BYTE      DPH1
      000000AEH   SFRSYM    DATA     BYTE      P1AL
      0000009AH   SFRSYM    DATA     BYTE      IEN2
      000000C0H   SFRSYM    DATA     BYTE      P2AL
      000000B6H   SFRSYM    DATA     BYTE      ADCDR0
      000000F8H.5 SFRSYM    DATA     BIT       RC16MF
      000000B7H   SFRSYM    DATA     BYTE      ADCDR1
      00000084H   SFRSYM    DATA     BYTE      DPL1
      000000D6H   SFRSYM    DATA     BYTE      P0OD
      000000DBH   SFRSYM    DATA     BYTE      P1OD
      000000D5H   SFRSYM    DATA     BYTE      P0PD
LX51 LINKER/LOCATER V4.66.97.0                                                        07/19/2022  10:30:28  PAGE 10


      00000098H.4 SFRSYM    DATA     BIT       REN0
      000000ECH   SFRSYM    DATA     BYTE      P2OD
      000000DAH   SFRSYM    DATA     BYTE      P1PD
      000000E4H   SFRSYM    DATA     BYTE      P2PD
      000000D7H   SFRSYM    DATA     BYTE      P0CS
      00000097H   SFRSYM    DATA     BYTE      P0DR
      0000009EH   SFRSYM    DATA     BYTE      EUARTEN
      000000DCH   SFRSYM    DATA     BYTE      P1CS
      000000E5H   SFRSYM    DATA     BYTE      P1DR
      000000F4H   SFRSYM    DATA     BYTE      P2CS
      000000FCH   SFRSYM    DATA     BYTE      P2DR
      000000D0H.7 SFRSYM    DATA     BIT       CY
      000000D8H.0 SFRSYM    DATA     BIT       WDT0
      000000D8H.1 SFRSYM    DATA     BIT       WDT1
      000000D8H.2 SFRSYM    DATA     BIT       WDT2
      00000081H   SFRSYM    DATA     BYTE      SP
      000000F1H   SFRSYM    DATA     BYTE      P0PU
      000000F2H   SFRSYM    DATA     BYTE      P1PU
      000000D1H   SFRSYM    DATA     WORD      OADR
      000000F3H   SFRSYM    DATA     BYTE      P2PU
      00000093H   SFRSYM    DATA     BYTE      ADCIER
      000000A5H   SFRSYM    DATA     BYTE      OSEC
      000000D8H.6 SFRSYM    DATA     BIT       WDEN
      000000BAH   SFRSYM    DATA     BYTE      S0RELH
      00000080H.0 SFRSYM    DATA     BIT       P00
      000000D8H.7 SFRSYM    DATA     BIT       WDOF
      000000BBH   SFRSYM    DATA     BYTE      S1RELH
      00000090H.0 SFRSYM    DATA     BIT       P10
      00000080H.1 SFRSYM    DATA     BIT       P01
      00000087H   SFRSYM    DATA     BYTE      PCON
      000000C4H   SFRSYM    DATA     BYTE      PWM0DH
      000000A0H.0 SFRSYM    DATA     BIT       P20
      00000090H.1 SFRSYM    DATA     BIT       P11
      00000080H.2 SFRSYM    DATA     BIT       P02
      000000C6H   SFRSYM    DATA     BYTE      PWM1DH
      00000090H.2 SFRSYM    DATA     BIT       P12
      00000080H.3 SFRSYM    DATA     BIT       P03
      000000C7H   SFRSYM    DATA     BYTE      PWM2DH
      000000C8H.2 SFRSYM    DATA     BIT       PWM0IE
      000000AAH   SFRSYM    DATA     BYTE      S0RELL
      000000A0H.2 SFRSYM    DATA     BIT       P22
      00000090H.3 SFRSYM    DATA     BIT       P13
      00000080H.4 SFRSYM    DATA     BIT       P04
      000000C8H.1 SFRSYM    DATA     BIT       PWM0IF
      0000009DH   SFRSYM    DATA     BYTE      S1RELL
      000000A0H.3 SFRSYM    DATA     BIT       P23
      00000090H.4 SFRSYM    DATA     BIT       P14
      00000080H.5 SFRSYM    DATA     BIT       P05
      000000C3H   SFRSYM    DATA     BYTE      PWM0DL
      00000090H.5 SFRSYM    DATA     BIT       P15
      000000A6H   SFRSYM    DATA     BYTE      OSTATUS
      000000C5H   SFRSYM    DATA     BYTE      PWM1DL
      000000A0H.5 SFRSYM    DATA     BIT       P25
      000000D8H.4 SFRSYM    DATA     BIT       PORF
      000000D8H   SFRSYM    DATA     BYTE      RSTSTAT
      000000CFH   SFRSYM    DATA     BYTE      PWM2DL
      000000A0H.6 SFRSYM    DATA     BIT       P26
      000000C8H.7 SFRSYM    DATA     BIT       PWM0EN
      000000A0H.7 SFRSYM    DATA     BIT       P27
      000000A8H.5 SFRSYM    DATA     BIT       EPWM
      000000D8H.5 SFRSYM    DATA     BIT       LVRF
      000000F8H   SFRSYM    DATA     BYTE      CLKCON
      000000CCH   SFRSYM    DATA     BYTE      PWM0PH
      000000CEH   SFRSYM    DATA     BYTE      PWM1PH
      000000B8H.5 SFRSYM    DATA     BIT       I2CINTEN
LX51 LINKER/LOCATER V4.66.97.0                                                        07/19/2022  10:30:28  PAGE 11


      000000C2H   SFRSYM    DATA     BYTE      PWM2PH
      000000F0H   SFRSYM    DATA     BYTE      B
      000000EEH   SFRSYM    DATA     BYTE      RCHDIV
      000000CBH   SFRSYM    DATA     BYTE      PWM0PL
      000000CDH   SFRSYM    DATA     BYTE      PWM1PL
      000000C1H   SFRSYM    DATA     BYTE      PWM2PL
      000000F7H   SFRSYM    DATA     BYTE      ADCSPW
      000000F8H.1 SFRSYM    DATA     BIT       XCLKEN
      000000E0H   SFRSYM    DATA     BYTE      ACC
      000000DDH   SFRSYM    DATA     BYTE      LVDCON
      000000A8H.4 SFRSYM    DATA     BIT       ES0
      000000A9H   SFRSYM    DATA     BYTE      IP0
      000000A8H.1 SFRSYM    DATA     BIT       ET0
      000000A8H.2 SFRSYM    DATA     BIT       ES1
      000000F6H   SFRSYM    DATA     BYTE      ADCCSTAT
      000000B9H   SFRSYM    DATA     BYTE      IP1
      000000A8H.3 SFRSYM    DATA     BIT       ET1
      00000098H.0 SFRSYM    DATA     BIT       RI0
      000000C8H.0 SFRSYM    DATA     BIT       PWM0SS
      00000098H.1 SFRSYM    DATA     BIT       TI0
      000000A8H.0 SFRSYM    DATA     BIT       EX0
      000000D0H.0 SFRSYM    DATA     BIT       P
      000000B8H.3 SFRSYM    DATA     BIT       EFCINTEN
      000000A2H   SFRSYM    DATA     BYTE      OINTEN
      00000098H.7 SFRSYM    DATA     BIT       SM0
      00000098H.6 SFRSYM    DATA     BIT       SM1
      000000FEH   SFRSYM    DATA     BYTE      ADCCDR0
      000000FFH   SFRSYM    DATA     BYTE      ADCCDR1
      000000D0H.3 SFRSYM    DATA     BIT       RS0
      000000ACH   SFRSYM    DATA     BYTE      ADCGCR0
      000000D0H.4 SFRSYM    DATA     BIT       RS1
      000000ADH   SFRSYM    DATA     BYTE      ADCGCR1
      000000B4H   SFRSYM    DATA     BYTE      ADCGCR2
      000000B5H   SFRSYM    DATA     BYTE      ADCGCR3
      000000F8H.3 SFRSYM    DATA     BIT       RC32KEN
      000000DEH   SFRSYM    DATA     BYTE      PCLK0
      000000DFH   SFRSYM    DATA     BYTE      PCLK1
      00000083H   SFRSYM    DATA     BYTE      DPH
      000000E9H   SFRSYM    DATA     BYTE      P0IEN
      000000F5H   SFRSYM    DATA     BYTE      ADCHL
      000000F8H.2 SFRSYM    DATA     BIT       RC16MEN
      000000EAH   SFRSYM    DATA     BYTE      P1IEN
      000000EBH   SFRSYM    DATA     BYTE      P2IEN
      000000B6H   SFRSYM    DATA     WORD      ADCDR
      000000B3H   SFRSYM    DATA     BYTE      XTHCTR
      00000082H   SFRSYM    DATA     BYTE      DPL
      00000099H   SFRSYM    DATA     BYTE      S0BUF
      0000009CH   SFRSYM    DATA     BYTE      S1BUF
      000000F9H   SFRSYM    DATA     BYTE      P0OEN
      000000B8H.0 SFRSYM    DATA     BIT       GTIM0INTEN
      000000D9H   SFRSYM    DATA     BYTE      SYSDIV
      00000098H   SFRSYM    DATA     BYTE      S0CON
      000000FAH   SFRSYM    DATA     BYTE      P1OEN
      000000B8H.2 SFRSYM    DATA     BIT       GTIM1INTEN
      000000A3H   SFRSYM    DATA     BYTE      OINTUS
      000000BEH   SFRSYM    DATA     BYTE      RCHTRIMH
      000000F8H.0 SFRSYM    DATA     BIT       SYSSEL
      0000009BH   SFRSYM    DATA     BYTE      S1CON
      000000FBH   SFRSYM    DATA     BYTE      P2OEN
      000000B8H.6 SFRSYM    DATA     BIT       GTIM2INTEN
      000000BDH   SFRSYM    DATA     BYTE      LDOTRIMH
      00000092H   SFRSYM    DATA     BYTE      DPS
      0000009FH   SFRSYM    DATA     BYTE      RCLTRIMH
      000000BFH   SFRSYM    DATA     BYTE      RCHTRIML
      000000D3H   SFRSYM    DATA     BYTE      ODATA
LX51 LINKER/LOCATER V4.66.97.0                                                        07/19/2022  10:30:28  PAGE 12


      00000091H   SFRSYM    DATA     BYTE      LDOTRIML
      000000BCH   SFRSYM    DATA     BYTE      RCLTRIML
      000000E1H   SFRSYM    DATA     BYTE      P0IRQ
      000000B8H.1 SFRSYM    DATA     BIT       SPIINTEN
      000000E2H   SFRSYM    DATA     BYTE      P1IRQ
      000000E3H   SFRSYM    DATA     BYTE      P2IRQ
      000000D2H   SFRSYM    DATA     BYTE      OADRH
      000000B8H.7 SFRSYM    DATA     BIT       UART2INTEN
      000000F0H.0 SFRSYM    DATA     BIT       B0
      000000F0H.1 SFRSYM    DATA     BIT       B1
      000000F0H.2 SFRSYM    DATA     BIT       B2
      000000D1H   SFRSYM    DATA     BYTE      OADRL
      000000F0H.3 SFRSYM    DATA     BIT       B3
      000000F0H.4 SFRSYM    DATA     BIT       B4
      000000D0H.5 SFRSYM    DATA     BIT       F0
      000000F0H.5 SFRSYM    DATA     BIT       B5
      000000D0H.1 SFRSYM    DATA     BIT       F1
      000000AFH   SFRSYM    DATA     BYTE      REMAP
      000000F0H.6 SFRSYM    DATA     BIT       B6
      000000E0H.0 SFRSYM    DATA     BIT       ACC0
      000000A1H   SFRSYM    DATA     BYTE      OUS
      000000C8H.6 SFRSYM    DATA     BIT       PWM0S
      000000F0H.7 SFRSYM    DATA     BIT       B7
      000000E0H.1 SFRSYM    DATA     BIT       ACC1
      000000F8H.4 SFRSYM    DATA     BIT       XCLKF
      000000E0H.2 SFRSYM    DATA     BIT       ACC2
      0000008EH   SFRSYM    DATA     BYTE      PDSEL
      000000E0H.3 SFRSYM    DATA     BIT       ACC3
      000000D0H   SFRSYM    DATA     BYTE      PSW
      000000E0H.4 SFRSYM    DATA     BIT       ACC4
      00000098H.2 SFRSYM    DATA     BIT       RB80
      000000E0H.5 SFRSYM    DATA     BIT       ACC5
      000000FDH   SFRSYM    DATA     BYTE      ADCVREF
      000000E0H.6 SFRSYM    DATA     BIT       ACC6

      01000710H   BLOCK     CODE     ---       LVL=0
      02000045H   SYMBOL    XDATA    DWORD     system_clk_hz
      01000716H   BLOCK     CODE     NEAR LAB  LVL=1
      02000049H   SYMBOL    XDATA    DWORD     crystal_clk
      ---         BLOCKEND  ---      ---       LVL=1
      01000710H   LINE      CODE     ---       #26
      01000716H   LINE      CODE     ---       #27
      01000716H   LINE      CODE     ---       #28
      01000720H   LINE      CODE     ---       #29
      01000723H   LINE      CODE     ---       #30
      0100072BH   LINE      CODE     ---       #33
      01000793H   LINE      CODE     ---       #38
      010007BBH   LINE      CODE     ---       #39
      010007BBH   LINE      CODE     ---       #40
      010007BBH   LINE      CODE     ---       #41
      010007BDH   LINE      CODE     ---       #42
      010007CFH   LINE      CODE     ---       #43
      010007CFH   LINE      CODE     ---       #44
      010007D9H   LINE      CODE     ---       #45
      010007DBH   LINE      CODE     ---       #47
      010007DBH   LINE      CODE     ---       #48
      010007F0H   LINE      CODE     ---       #49
      010007F0H   LINE      CODE     ---       #50
      0100080FH   LINE      CODE     ---       #51
      0100080FH   LINE      CODE     ---       #52
      0100080FH   LINE      CODE     ---       #53
      01000812H   LINE      CODE     ---       #54
      01000815H   LINE      CODE     ---       #55
      01000817H   LINE      CODE     ---       #56
      01000817H   LINE      CODE     ---       #57
LX51 LINKER/LOCATER V4.66.97.0                                                        07/19/2022  10:30:28  PAGE 13


      0100081AH   LINE      CODE     ---       #58
      0100081DH   LINE      CODE     ---       #59
      0100081FH   LINE      CODE     ---       #60
      0100081FH   LINE      CODE     ---       #61
      01000822H   LINE      CODE     ---       #62
      01000825H   LINE      CODE     ---       #63
      01000825H   LINE      CODE     ---       #64
      01000837H   LINE      CODE     ---       #67
      01000837H   LINE      CODE     ---       #69
      01000837H   LINE      CODE     ---       #71
      0100083AH   LINE      CODE     ---       #72
      0100083DH   LINE      CODE     ---       #73
      ---         BLOCKEND  ---      ---       LVL=0

      0100004DH   BLOCK     CODE     ---       LVL=0
      0100004DH   LINE      CODE     ---       #82
      0100004DH   LINE      CODE     ---       #83
      0100004DH   LINE      CODE     ---       #84
      ---         BLOCKEND  ---      ---       LVL=0

      ---         MODULE    ---      ---       COMMON
      00000098H.3 SFRSYM    DATA     BIT       TB80
      000000E0H.7 SFRSYM    DATA     BIT       ACC7
      00000080H   SFRSYM    DATA     BYTE      P0
      00000090H   SFRSYM    DATA     BYTE      P1
      000000A0H   SFRSYM    DATA     BYTE      P2
      00000098H.5 SFRSYM    DATA     BIT       SM20
      000000B2H   SFRSYM    DATA     BYTE      ESTCR
      000000B1H   SFRSYM    DATA     BYTE      CLKST
      000000D0H.6 SFRSYM    DATA     BIT       AC
      000000D8H.3 SFRSYM    DATA     BIT       ERSTF
      000000E6H   SFRSYM    DATA     BYTE      PRESET0
      000000D4H   SFRSYM    DATA     BYTE      OCTRL
      000000A8H.7 SFRSYM    DATA     BIT       EA
      0000008FH   SFRSYM    DATA     BYTE      POREN
      000000C8H   SFRSYM    DATA     BYTE      PWM0CON
      000000E7H   SFRSYM    DATA     BYTE      PRESET1
      000000C9H   SFRSYM    DATA     BYTE      PWM1CON
      00000086H   SFRSYM    DATA     BYTE      BEEPCTR
      000000CAH   SFRSYM    DATA     BYTE      PWM2CON
      000000B8H.4 SFRSYM    DATA     BIT       LPTIMINTEN
      000000ABH   SFRSYM    DATA     BYTE      P0AH
      000000B0H   SFRSYM    DATA     BYTE      P1AH
      000000E8H   SFRSYM    DATA     BYTE      P2AH
      000000F8H.6 SFRSYM    DATA     BIT       RC32KF
      000000A8H   SFRSYM    DATA     BYTE      IEN0
      000000A7H   SFRSYM    DATA     BYTE      OPSET
      000000A4H   SFRSYM    DATA     BYTE      P0AL
      000000B8H   SFRSYM    DATA     BYTE      IEN1
      000000A8H.6 SFRSYM    DATA     BIT       EADC
      00000085H   SFRSYM    DATA     BYTE      DPH1
      000000AEH   SFRSYM    DATA     BYTE      P1AL
      0000009AH   SFRSYM    DATA     BYTE      IEN2
      000000C0H   SFRSYM    DATA     BYTE      P2AL
      000000B6H   SFRSYM    DATA     BYTE      ADCDR0
      000000F8H.5 SFRSYM    DATA     BIT       RC16MF
      000000B7H   SFRSYM    DATA     BYTE      ADCDR1
      00000084H   SFRSYM    DATA     BYTE      DPL1
      000000D6H   SFRSYM    DATA     BYTE      P0OD
      000000DBH   SFRSYM    DATA     BYTE      P1OD
      000000D5H   SFRSYM    DATA     BYTE      P0PD
      00000098H.4 SFRSYM    DATA     BIT       REN0
      000000ECH   SFRSYM    DATA     BYTE      P2OD
      000000DAH   SFRSYM    DATA     BYTE      P1PD
      000000E4H   SFRSYM    DATA     BYTE      P2PD
LX51 LINKER/LOCATER V4.66.97.0                                                        07/19/2022  10:30:28  PAGE 14


      000000D7H   SFRSYM    DATA     BYTE      P0CS
      00000097H   SFRSYM    DATA     BYTE      P0DR
      0000009EH   SFRSYM    DATA     BYTE      EUARTEN
      000000DCH   SFRSYM    DATA     BYTE      P1CS
      000000E5H   SFRSYM    DATA     BYTE      P1DR
      000000F4H   SFRSYM    DATA     BYTE      P2CS
      000000FCH   SFRSYM    DATA     BYTE      P2DR
      000000D0H.7 SFRSYM    DATA     BIT       CY
      000000D8H.0 SFRSYM    DATA     BIT       WDT0
      000000D8H.1 SFRSYM    DATA     BIT       WDT1
      000000D8H.2 SFRSYM    DATA     BIT       WDT2
      00000081H   SFRSYM    DATA     BYTE      SP
      000000F1H   SFRSYM    DATA     BYTE      P0PU
      000000F2H   SFRSYM    DATA     BYTE      P1PU
      000000D1H   SFRSYM    DATA     WORD      OADR
      000000F3H   SFRSYM    DATA     BYTE      P2PU
      00000093H   SFRSYM    DATA     BYTE      ADCIER
      000000A5H   SFRSYM    DATA     BYTE      OSEC
      000000D8H.6 SFRSYM    DATA     BIT       WDEN
      000000BAH   SFRSYM    DATA     BYTE      S0RELH
      00000080H.0 SFRSYM    DATA     BIT       P00
      000000D8H.7 SFRSYM    DATA     BIT       WDOF
      000000BBH   SFRSYM    DATA     BYTE      S1RELH
      00000090H.0 SFRSYM    DATA     BIT       P10
      00000080H.1 SFRSYM    DATA     BIT       P01
      00000087H   SFRSYM    DATA     BYTE      PCON
      000000C4H   SFRSYM    DATA     BYTE      PWM0DH
      000000A0H.0 SFRSYM    DATA     BIT       P20
      00000090H.1 SFRSYM    DATA     BIT       P11
      00000080H.2 SFRSYM    DATA     BIT       P02
      000000C6H   SFRSYM    DATA     BYTE      PWM1DH
      00000090H.2 SFRSYM    DATA     BIT       P12
      00000080H.3 SFRSYM    DATA     BIT       P03
      000000C7H   SFRSYM    DATA     BYTE      PWM2DH
      000000C8H.2 SFRSYM    DATA     BIT       PWM0IE
      000000AAH   SFRSYM    DATA     BYTE      S0RELL
      000000A0H.2 SFRSYM    DATA     BIT       P22
      00000090H.3 SFRSYM    DATA     BIT       P13
      00000080H.4 SFRSYM    DATA     BIT       P04
      000000C8H.1 SFRSYM    DATA     BIT       PWM0IF
      0000009DH   SFRSYM    DATA     BYTE      S1RELL
      000000A0H.3 SFRSYM    DATA     BIT       P23
      00000090H.4 SFRSYM    DATA     BIT       P14
      00000080H.5 SFRSYM    DATA     BIT       P05
      000000C3H   SFRSYM    DATA     BYTE      PWM0DL
      00000090H.5 SFRSYM    DATA     BIT       P15
      000000A6H   SFRSYM    DATA     BYTE      OSTATUS
      000000C5H   SFRSYM    DATA     BYTE      PWM1DL
      000000A0H.5 SFRSYM    DATA     BIT       P25
      000000D8H.4 SFRSYM    DATA     BIT       PORF
      000000D8H   SFRSYM    DATA     BYTE      RSTSTAT
      000000CFH   SFRSYM    DATA     BYTE      PWM2DL
      000000A0H.6 SFRSYM    DATA     BIT       P26
      000000C8H.7 SFRSYM    DATA     BIT       PWM0EN
      000000A0H.7 SFRSYM    DATA     BIT       P27
      000000A8H.5 SFRSYM    DATA     BIT       EPWM
      000000D8H.5 SFRSYM    DATA     BIT       LVRF
      000000F8H   SFRSYM    DATA     BYTE      CLKCON
      000000CCH   SFRSYM    DATA     BYTE      PWM0PH
      000000CEH   SFRSYM    DATA     BYTE      PWM1PH
      000000B8H.5 SFRSYM    DATA     BIT       I2CINTEN
      000000C2H   SFRSYM    DATA     BYTE      PWM2PH
      000000F0H   SFRSYM    DATA     BYTE      B
      000000EEH   SFRSYM    DATA     BYTE      RCHDIV
      000000CBH   SFRSYM    DATA     BYTE      PWM0PL
LX51 LINKER/LOCATER V4.66.97.0                                                        07/19/2022  10:30:28  PAGE 15


      000000CDH   SFRSYM    DATA     BYTE      PWM1PL
      000000C1H   SFRSYM    DATA     BYTE      PWM2PL
      000000F7H   SFRSYM    DATA     BYTE      ADCSPW
      000000F8H.1 SFRSYM    DATA     BIT       XCLKEN
      000000E0H   SFRSYM    DATA     BYTE      ACC
      000000DDH   SFRSYM    DATA     BYTE      LVDCON
      000000A8H.4 SFRSYM    DATA     BIT       ES0
      000000A9H   SFRSYM    DATA     BYTE      IP0
      000000A8H.1 SFRSYM    DATA     BIT       ET0
      000000A8H.2 SFRSYM    DATA     BIT       ES1
      000000F6H   SFRSYM    DATA     BYTE      ADCCSTAT
      000000B9H   SFRSYM    DATA     BYTE      IP1
      000000A8H.3 SFRSYM    DATA     BIT       ET1
      00000098H.0 SFRSYM    DATA     BIT       RI0
      000000C8H.0 SFRSYM    DATA     BIT       PWM0SS
      00000098H.1 SFRSYM    DATA     BIT       TI0
      000000A8H.0 SFRSYM    DATA     BIT       EX0
      000000D0H.0 SFRSYM    DATA     BIT       P
      000000B8H.3 SFRSYM    DATA     BIT       EFCINTEN
      000000A2H   SFRSYM    DATA     BYTE      OINTEN
      00000098H.7 SFRSYM    DATA     BIT       SM0
      00000098H.6 SFRSYM    DATA     BIT       SM1
      000000FEH   SFRSYM    DATA     BYTE      ADCCDR0
      000000FFH   SFRSYM    DATA     BYTE      ADCCDR1
      000000D0H.3 SFRSYM    DATA     BIT       RS0
      000000ACH   SFRSYM    DATA     BYTE      ADCGCR0
      000000D0H.4 SFRSYM    DATA     BIT       RS1
      000000ADH   SFRSYM    DATA     BYTE      ADCGCR1
      000000B4H   SFRSYM    DATA     BYTE      ADCGCR2
      000000B5H   SFRSYM    DATA     BYTE      ADCGCR3
      000000F8H.3 SFRSYM    DATA     BIT       RC32KEN
      000000DEH   SFRSYM    DATA     BYTE      PCLK0
      000000DFH   SFRSYM    DATA     BYTE      PCLK1
      00000083H   SFRSYM    DATA     BYTE      DPH
      000000E9H   SFRSYM    DATA     BYTE      P0IEN
      000000F5H   SFRSYM    DATA     BYTE      ADCHL
      000000F8H.2 SFRSYM    DATA     BIT       RC16MEN
      000000EAH   SFRSYM    DATA     BYTE      P1IEN
      000000EBH   SFRSYM    DATA     BYTE      P2IEN
      000000B6H   SFRSYM    DATA     WORD      ADCDR
      000000B3H   SFRSYM    DATA     BYTE      XTHCTR
      00000082H   SFRSYM    DATA     BYTE      DPL
      00000099H   SFRSYM    DATA     BYTE      S0BUF
      0000009CH   SFRSYM    DATA     BYTE      S1BUF
      000000F9H   SFRSYM    DATA     BYTE      P0OEN
      000000B8H.0 SFRSYM    DATA     BIT       GTIM0INTEN
      000000D9H   SFRSYM    DATA     BYTE      SYSDIV
      00000098H   SFRSYM    DATA     BYTE      S0CON
      000000FAH   SFRSYM    DATA     BYTE      P1OEN
      000000B8H.2 SFRSYM    DATA     BIT       GTIM1INTEN
      000000A3H   SFRSYM    DATA     BYTE      OINTUS
      000000BEH   SFRSYM    DATA     BYTE      RCHTRIMH
      000000F8H.0 SFRSYM    DATA     BIT       SYSSEL
      0000009BH   SFRSYM    DATA     BYTE      S1CON
      000000FBH   SFRSYM    DATA     BYTE      P2OEN
      000000B8H.6 SFRSYM    DATA     BIT       GTIM2INTEN
      000000BDH   SFRSYM    DATA     BYTE      LDOTRIMH
      00000092H   SFRSYM    DATA     BYTE      DPS
      0000009FH   SFRSYM    DATA     BYTE      RCLTRIMH
      000000BFH   SFRSYM    DATA     BYTE      RCHTRIML
      000000D3H   SFRSYM    DATA     BYTE      ODATA
      00000091H   SFRSYM    DATA     BYTE      LDOTRIML
      000000BCH   SFRSYM    DATA     BYTE      RCLTRIML
      000000E1H   SFRSYM    DATA     BYTE      P0IRQ
      000000B8H.1 SFRSYM    DATA     BIT       SPIINTEN
LX51 LINKER/LOCATER V4.66.97.0                                                        07/19/2022  10:30:28  PAGE 16


      000000E2H   SFRSYM    DATA     BYTE      P1IRQ
      000000E3H   SFRSYM    DATA     BYTE      P2IRQ
      000000D2H   SFRSYM    DATA     BYTE      OADRH
      000000B8H.7 SFRSYM    DATA     BIT       UART2INTEN
      000000F0H.0 SFRSYM    DATA     BIT       B0
      000000F0H.1 SFRSYM    DATA     BIT       B1
      000000F0H.2 SFRSYM    DATA     BIT       B2
      000000D1H   SFRSYM    DATA     BYTE      OADRL
      000000F0H.3 SFRSYM    DATA     BIT       B3
      000000F0H.4 SFRSYM    DATA     BIT       B4
      000000D0H.5 SFRSYM    DATA     BIT       F0
      000000F0H.5 SFRSYM    DATA     BIT       B5
      000000D0H.1 SFRSYM    DATA     BIT       F1
      000000AFH   SFRSYM    DATA     BYTE      REMAP
      000000F0H.6 SFRSYM    DATA     BIT       B6
      000000E0H.0 SFRSYM    DATA     BIT       ACC0
      000000A1H   SFRSYM    DATA     BYTE      OUS
      000000C8H.6 SFRSYM    DATA     BIT       PWM0S
      000000F0H.7 SFRSYM    DATA     BIT       B7
      000000E0H.1 SFRSYM    DATA     BIT       ACC1
      000000F8H.4 SFRSYM    DATA     BIT       XCLKF
      000000E0H.2 SFRSYM    DATA     BIT       ACC2
      0000008EH   SFRSYM    DATA     BYTE      PDSEL
      000000E0H.3 SFRSYM    DATA     BIT       ACC3
      000000D0H   SFRSYM    DATA     BYTE      PSW
      000000E0H.4 SFRSYM    DATA     BIT       ACC4
      00000098H.2 SFRSYM    DATA     BIT       RB80
      000000E0H.5 SFRSYM    DATA     BIT       ACC5
      000000FDH   SFRSYM    DATA     BYTE      ADCVREF
      000000E0H.6 SFRSYM    DATA     BIT       ACC6
      00000007H   SYMBOL    DATA     BYTE      i
      00000006H   SYMBOL    DATA     BYTE      j

      ---         MODULE    ---      ---       UART0
      02000076H   PUBLIC    XDATA    ---       uart0_func
      02000075H   PUBLIC    XDATA    BYTE      tx_flag
      01000A7BH   PUBLIC    CODE     ---       _putchar
      01000058H   PUBLIC    CODE     ---       uart0_recv_byte
      01000A36H   PUBLIC    CODE     ---       _uart0_send_byte
      01000A4CH   PUBLIC    CODE     ---       _uart0_irq_init
      010009C4H   PUBLIC    CODE     ---       _uart0_init
      01000941H   PUBLIC    CODE     ---       UART0_IRQHandler
      00000098H.3 SFRSYM    DATA     BIT       TB80
      000000E0H.7 SFRSYM    DATA     BIT       ACC7
      00000080H   SFRSYM    DATA     BYTE      P0
      00000090H   SFRSYM    DATA     BYTE      P1
      000000A0H   SFRSYM    DATA     BYTE      P2
      00000098H.5 SFRSYM    DATA     BIT       SM20
      000000B2H   SFRSYM    DATA     BYTE      ESTCR
      000000B1H   SFRSYM    DATA     BYTE      CLKST
      000000D0H.6 SFRSYM    DATA     BIT       AC
      000000D8H.3 SFRSYM    DATA     BIT       ERSTF
      000000E6H   SFRSYM    DATA     BYTE      PRESET0
      000000D4H   SFRSYM    DATA     BYTE      OCTRL
      000000A8H.7 SFRSYM    DATA     BIT       EA
      0000008FH   SFRSYM    DATA     BYTE      POREN
      000000C8H   SFRSYM    DATA     BYTE      PWM0CON
      000000E7H   SFRSYM    DATA     BYTE      PRESET1
      000000C9H   SFRSYM    DATA     BYTE      PWM1CON
      00000086H   SFRSYM    DATA     BYTE      BEEPCTR
      000000CAH   SFRSYM    DATA     BYTE      PWM2CON
      000000B8H.4 SFRSYM    DATA     BIT       LPTIMINTEN
      000000ABH   SFRSYM    DATA     BYTE      P0AH
      000000B0H   SFRSYM    DATA     BYTE      P1AH
      000000E8H   SFRSYM    DATA     BYTE      P2AH
LX51 LINKER/LOCATER V4.66.97.0                                                        07/19/2022  10:30:28  PAGE 17


      000000F8H.6 SFRSYM    DATA     BIT       RC32KF
      000000A8H   SFRSYM    DATA     BYTE      IEN0
      000000A7H   SFRSYM    DATA     BYTE      OPSET
      000000A4H   SFRSYM    DATA     BYTE      P0AL
      000000B8H   SFRSYM    DATA     BYTE      IEN1
      000000A8H.6 SFRSYM    DATA     BIT       EADC
      00000085H   SFRSYM    DATA     BYTE      DPH1
      000000AEH   SFRSYM    DATA     BYTE      P1AL
      0000009AH   SFRSYM    DATA     BYTE      IEN2
      000000C0H   SFRSYM    DATA     BYTE      P2AL
      000000B6H   SFRSYM    DATA     BYTE      ADCDR0
      000000F8H.5 SFRSYM    DATA     BIT       RC16MF
      000000B7H   SFRSYM    DATA     BYTE      ADCDR1
      00000084H   SFRSYM    DATA     BYTE      DPL1
      000000D6H   SFRSYM    DATA     BYTE      P0OD
      000000DBH   SFRSYM    DATA     BYTE      P1OD
      000000D5H   SFRSYM    DATA     BYTE      P0PD
      00000098H.4 SFRSYM    DATA     BIT       REN0
      000000ECH   SFRSYM    DATA     BYTE      P2OD
      000000DAH   SFRSYM    DATA     BYTE      P1PD
      000000E4H   SFRSYM    DATA     BYTE      P2PD
      000000D7H   SFRSYM    DATA     BYTE      P0CS
      00000097H   SFRSYM    DATA     BYTE      P0DR
      0000009EH   SFRSYM    DATA     BYTE      EUARTEN
      000000DCH   SFRSYM    DATA     BYTE      P1CS
      000000E5H   SFRSYM    DATA     BYTE      P1DR
      000000F4H   SFRSYM    DATA     BYTE      P2CS
      000000FCH   SFRSYM    DATA     BYTE      P2DR
      000000D0H.7 SFRSYM    DATA     BIT       CY
      000000D8H.0 SFRSYM    DATA     BIT       WDT0
      000000D8H.1 SFRSYM    DATA     BIT       WDT1
      000000D8H.2 SFRSYM    DATA     BIT       WDT2
      00000081H   SFRSYM    DATA     BYTE      SP
      000000F1H   SFRSYM    DATA     BYTE      P0PU
      000000F2H   SFRSYM    DATA     BYTE      P1PU
      000000D1H   SFRSYM    DATA     WORD      OADR
      000000F3H   SFRSYM    DATA     BYTE      P2PU
      00000093H   SFRSYM    DATA     BYTE      ADCIER
      000000A5H   SFRSYM    DATA     BYTE      OSEC
      000000D8H.6 SFRSYM    DATA     BIT       WDEN
      000000BAH   SFRSYM    DATA     BYTE      S0RELH
      00000080H.0 SFRSYM    DATA     BIT       P00
      000000D8H.7 SFRSYM    DATA     BIT       WDOF
      000000BBH   SFRSYM    DATA     BYTE      S1RELH
      00000090H.0 SFRSYM    DATA     BIT       P10
      00000080H.1 SFRSYM    DATA     BIT       P01
      00000087H   SFRSYM    DATA     BYTE      PCON
      000000C4H   SFRSYM    DATA     BYTE      PWM0DH
      000000A0H.0 SFRSYM    DATA     BIT       P20
      00000090H.1 SFRSYM    DATA     BIT       P11
      00000080H.2 SFRSYM    DATA     BIT       P02
      000000C6H   SFRSYM    DATA     BYTE      PWM1DH
      00000090H.2 SFRSYM    DATA     BIT       P12
      00000080H.3 SFRSYM    DATA     BIT       P03
      000000C7H   SFRSYM    DATA     BYTE      PWM2DH
      000000C8H.2 SFRSYM    DATA     BIT       PWM0IE
      000000AAH   SFRSYM    DATA     BYTE      S0RELL
      000000A0H.2 SFRSYM    DATA     BIT       P22
      00000090H.3 SFRSYM    DATA     BIT       P13
      00000080H.4 SFRSYM    DATA     BIT       P04
      000000C8H.1 SFRSYM    DATA     BIT       PWM0IF
      0000009DH   SFRSYM    DATA     BYTE      S1RELL
      000000A0H.3 SFRSYM    DATA     BIT       P23
      00000090H.4 SFRSYM    DATA     BIT       P14
      00000080H.5 SFRSYM    DATA     BIT       P05
LX51 LINKER/LOCATER V4.66.97.0                                                        07/19/2022  10:30:28  PAGE 18


      000000C3H   SFRSYM    DATA     BYTE      PWM0DL
      00000090H.5 SFRSYM    DATA     BIT       P15
      000000A6H   SFRSYM    DATA     BYTE      OSTATUS
      000000C5H   SFRSYM    DATA     BYTE      PWM1DL
      000000A0H.5 SFRSYM    DATA     BIT       P25
      000000D8H.4 SFRSYM    DATA     BIT       PORF
      000000D8H   SFRSYM    DATA     BYTE      RSTSTAT
      000000CFH   SFRSYM    DATA     BYTE      PWM2DL
      000000A0H.6 SFRSYM    DATA     BIT       P26
      000000C8H.7 SFRSYM    DATA     BIT       PWM0EN
      000000A0H.7 SFRSYM    DATA     BIT       P27
      000000A8H.5 SFRSYM    DATA     BIT       EPWM
      000000D8H.5 SFRSYM    DATA     BIT       LVRF
      000000F8H   SFRSYM    DATA     BYTE      CLKCON
      000000CCH   SFRSYM    DATA     BYTE      PWM0PH
      000000CEH   SFRSYM    DATA     BYTE      PWM1PH
      000000B8H.5 SFRSYM    DATA     BIT       I2CINTEN
      000000C2H   SFRSYM    DATA     BYTE      PWM2PH
      000000F0H   SFRSYM    DATA     BYTE      B
      000000EEH   SFRSYM    DATA     BYTE      RCHDIV
      000000CBH   SFRSYM    DATA     BYTE      PWM0PL
      000000CDH   SFRSYM    DATA     BYTE      PWM1PL
      000000C1H   SFRSYM    DATA     BYTE      PWM2PL
      000000F7H   SFRSYM    DATA     BYTE      ADCSPW
      000000F8H.1 SFRSYM    DATA     BIT       XCLKEN
      000000E0H   SFRSYM    DATA     BYTE      ACC
      000000DDH   SFRSYM    DATA     BYTE      LVDCON
      000000A8H.4 SFRSYM    DATA     BIT       ES0
      000000A9H   SFRSYM    DATA     BYTE      IP0
      000000A8H.1 SFRSYM    DATA     BIT       ET0
      000000A8H.2 SFRSYM    DATA     BIT       ES1
      000000F6H   SFRSYM    DATA     BYTE      ADCCSTAT
      000000B9H   SFRSYM    DATA     BYTE      IP1
      000000A8H.3 SFRSYM    DATA     BIT       ET1
      00000098H.0 SFRSYM    DATA     BIT       RI0
      000000C8H.0 SFRSYM    DATA     BIT       PWM0SS
      00000098H.1 SFRSYM    DATA     BIT       TI0
      000000A8H.0 SFRSYM    DATA     BIT       EX0
      000000D0H.0 SFRSYM    DATA     BIT       P
      000000B8H.3 SFRSYM    DATA     BIT       EFCINTEN
      000000A2H   SFRSYM    DATA     BYTE      OINTEN
      00000098H.7 SFRSYM    DATA     BIT       SM0
      00000098H.6 SFRSYM    DATA     BIT       SM1
      000000FEH   SFRSYM    DATA     BYTE      ADCCDR0
      000000FFH   SFRSYM    DATA     BYTE      ADCCDR1
      000000D0H.3 SFRSYM    DATA     BIT       RS0
      000000ACH   SFRSYM    DATA     BYTE      ADCGCR0
      000000D0H.4 SFRSYM    DATA     BIT       RS1
      000000ADH   SFRSYM    DATA     BYTE      ADCGCR1
      000000B4H   SFRSYM    DATA     BYTE      ADCGCR2
      000000B5H   SFRSYM    DATA     BYTE      ADCGCR3
      000000F8H.3 SFRSYM    DATA     BIT       RC32KEN
      000000DEH   SFRSYM    DATA     BYTE      PCLK0
      000000DFH   SFRSYM    DATA     BYTE      PCLK1
      00000083H   SFRSYM    DATA     BYTE      DPH
      000000E9H   SFRSYM    DATA     BYTE      P0IEN
      000000F5H   SFRSYM    DATA     BYTE      ADCHL
      000000F8H.2 SFRSYM    DATA     BIT       RC16MEN
      000000EAH   SFRSYM    DATA     BYTE      P1IEN
      000000EBH   SFRSYM    DATA     BYTE      P2IEN
      000000B6H   SFRSYM    DATA     WORD      ADCDR
      000000B3H   SFRSYM    DATA     BYTE      XTHCTR
      00000082H   SFRSYM    DATA     BYTE      DPL
      00000099H   SFRSYM    DATA     BYTE      S0BUF
      0000009CH   SFRSYM    DATA     BYTE      S1BUF
LX51 LINKER/LOCATER V4.66.97.0                                                        07/19/2022  10:30:28  PAGE 19


      000000F9H   SFRSYM    DATA     BYTE      P0OEN
      000000B8H.0 SFRSYM    DATA     BIT       GTIM0INTEN
      000000D9H   SFRSYM    DATA     BYTE      SYSDIV
      00000098H   SFRSYM    DATA     BYTE      S0CON
      000000FAH   SFRSYM    DATA     BYTE      P1OEN
      000000B8H.2 SFRSYM    DATA     BIT       GTIM1INTEN
      000000A3H   SFRSYM    DATA     BYTE      OINTUS
      000000BEH   SFRSYM    DATA     BYTE      RCHTRIMH
      000000F8H.0 SFRSYM    DATA     BIT       SYSSEL
      0000009BH   SFRSYM    DATA     BYTE      S1CON
      000000FBH   SFRSYM    DATA     BYTE      P2OEN
      000000B8H.6 SFRSYM    DATA     BIT       GTIM2INTEN
      000000BDH   SFRSYM    DATA     BYTE      LDOTRIMH
      00000092H   SFRSYM    DATA     BYTE      DPS
      0000009FH   SFRSYM    DATA     BYTE      RCLTRIMH
      000000BFH   SFRSYM    DATA     BYTE      RCHTRIML
      000000D3H   SFRSYM    DATA     BYTE      ODATA
      00000091H   SFRSYM    DATA     BYTE      LDOTRIML
      000000BCH   SFRSYM    DATA     BYTE      RCLTRIML
      000000E1H   SFRSYM    DATA     BYTE      P0IRQ
      000000B8H.1 SFRSYM    DATA     BIT       SPIINTEN
      000000E2H   SFRSYM    DATA     BYTE      P1IRQ
      000000E3H   SFRSYM    DATA     BYTE      P2IRQ
      000000D2H   SFRSYM    DATA     BYTE      OADRH
      000000B8H.7 SFRSYM    DATA     BIT       UART2INTEN
      000000F0H.0 SFRSYM    DATA     BIT       B0
      000000F0H.1 SFRSYM    DATA     BIT       B1
      000000F0H.2 SFRSYM    DATA     BIT       B2
      000000D1H   SFRSYM    DATA     BYTE      OADRL
      000000F0H.3 SFRSYM    DATA     BIT       B3
      000000F0H.4 SFRSYM    DATA     BIT       B4
      000000D0H.5 SFRSYM    DATA     BIT       F0
      000000F0H.5 SFRSYM    DATA     BIT       B5
      000000D0H.1 SFRSYM    DATA     BIT       F1
      000000AFH   SFRSYM    DATA     BYTE      REMAP
      000000F0H.6 SFRSYM    DATA     BIT       B6
      000000E0H.0 SFRSYM    DATA     BIT       ACC0
      000000A1H   SFRSYM    DATA     BYTE      OUS
      000000C8H.6 SFRSYM    DATA     BIT       PWM0S
      000000F0H.7 SFRSYM    DATA     BIT       B7
      000000E0H.1 SFRSYM    DATA     BIT       ACC1
      000000F8H.4 SFRSYM    DATA     BIT       XCLKF
      000000E0H.2 SFRSYM    DATA     BIT       ACC2
      0000008EH   SFRSYM    DATA     BYTE      PDSEL
      000000E0H.3 SFRSYM    DATA     BIT       ACC3
      000000D0H   SFRSYM    DATA     BYTE      PSW
      000000E0H.4 SFRSYM    DATA     BIT       ACC4
      00000098H.2 SFRSYM    DATA     BIT       RB80
      000000E0H.5 SFRSYM    DATA     BIT       ACC5
      000000FDH   SFRSYM    DATA     BYTE      ADCVREF
      000000E0H.6 SFRSYM    DATA     BIT       ACC6
      010008CAH   SYMBOL    CODE     ---       _uart0_set_baud_rate

      01000941H   BLOCK     CODE     ---       LVL=0
      01000941H   LINE      CODE     ---       #24
      0100095EH   LINE      CODE     ---       #26
      01000961H   LINE      CODE     ---       #27
      01000961H   LINE      CODE     ---       #28
      0100096BH   LINE      CODE     ---       #29
      0100096BH   LINE      CODE     ---       #30
      0100096EH   LINE      CODE     ---       #31
      0100096EH   LINE      CODE     ---       #32
      01000970H   LINE      CODE     ---       #33
      01000970H   LINE      CODE     ---       #42
      ---         BLOCKEND  ---      ---       LVL=0
LX51 LINKER/LOCATER V4.66.97.0                                                        07/19/2022  10:30:28  PAGE 20



      010008CAH   BLOCK     CODE     ---       LVL=0
      02000049H   SYMBOL    XDATA    DWORD     clk_hz
      0200004DH   SYMBOL    XDATA    DWORD     baud_rate
      010008D0H   BLOCK     CODE     NEAR LAB  LVL=1
      02000051H   SYMBOL    XDATA    DWORD     temp
      00000003H   SYMBOL    DATA     BYTE      MSbyte
      00000007H   SYMBOL    DATA     BYTE      LSbyte
      ---         BLOCKEND  ---      ---       LVL=1
      010008CAH   LINE      CODE     ---       #52
      010008D0H   LINE      CODE     ---       #53
      010008D0H   LINE      CODE     ---       #57
      010008E5H   LINE      CODE     ---       #58
      0100090CH   LINE      CODE     ---       #59
      01000926H   LINE      CODE     ---       #61
      01000933H   LINE      CODE     ---       #62
      01000939H   LINE      CODE     ---       #64
      0100093EH   LINE      CODE     ---       #65
      01000940H   LINE      CODE     ---       #66
      ---         BLOCKEND  ---      ---       LVL=0

      010009C4H   BLOCK     CODE     ---       LVL=0
      02000045H   SYMBOL    XDATA    DWORD     baud_rate
      010009C4H   LINE      CODE     ---       #75
      010009CAH   LINE      CODE     ---       #76
      010009CAH   LINE      CODE     ---       #78
      010009CDH   LINE      CODE     ---       #79
      010009D0H   LINE      CODE     ---       #80
      010009D3H   LINE      CODE     ---       #82
      010009D8H   LINE      CODE     ---       #84
      010009DAH   LINE      CODE     ---       #85
      010009DCH   LINE      CODE     ---       #87
      010009DEH   LINE      CODE     ---       #88
      010009E0H   LINE      CODE     ---       #90
      010009F5H   LINE      CODE     ---       #91
      010009F7H   LINE      CODE     ---       #93
      010009FAH   LINE      CODE     ---       #94
      ---         BLOCKEND  ---      ---       LVL=0

      01000A4CH   BLOCK     CODE     ---       LVL=0
      00000007H   SYMBOL    DATA     BYTE      irqstate
      00000001H   SYMBOL    DATA     ---       pfunc_recv
      01000A4CH   LINE      CODE     ---       #104
      01000A4CH   LINE      CODE     ---       #105
      01000A4CH   LINE      CODE     ---       #106
      01000A51H   LINE      CODE     ---       #107
      01000A51H   LINE      CODE     ---       #108
      01000A53H   LINE      CODE     ---       #109
      01000A55H   LINE      CODE     ---       #111
      01000A5BH   LINE      CODE     ---       #112
      01000A5BH   LINE      CODE     ---       #114
      01000A5BH   LINE      CODE     ---       #116
      01000A5DH   LINE      CODE     ---       #117
      01000A5DH   LINE      CODE     ---       #118
      ---         BLOCKEND  ---      ---       LVL=0

      01000A36H   BLOCK     CODE     ---       LVL=0
      00000007H   SYMBOL    DATA     CHAR      c
      01000A36H   BLOCK     CODE     NEAR LAB  LVL=1
      00000004H   SYMBOL    DATA     WORD      timeout
      ---         BLOCKEND  ---      ---       LVL=1
      01000A36H   LINE      CODE     ---       #127
      01000A36H   LINE      CODE     ---       #128
      01000A36H   LINE      CODE     ---       #131
      01000A3AH   LINE      CODE     ---       #133
LX51 LINKER/LOCATER V4.66.97.0                                                        07/19/2022  10:30:28  PAGE 21


      01000A3CH   LINE      CODE     ---       #140
      01000A3FH   LINE      CODE     ---       #141
      01000A3FH   LINE      CODE     ---       #142
      01000A49H   LINE      CODE     ---       #143
      01000A49H   LINE      CODE     ---       #144
      01000A49H   LINE      CODE     ---       #145
      01000A49H   LINE      CODE     ---       #146
      01000A49H   LINE      CODE     ---       #147
      01000A4BH   LINE      CODE     ---       #149
      ---         BLOCKEND  ---      ---       LVL=0

      01000058H   BLOCK     CODE     ---       LVL=0
      01000058H   LINE      CODE     ---       #174
      01000058H   LINE      CODE     ---       #175
      01000058H   LINE      CODE     ---       #176
      0100005AH   LINE      CODE     ---       #177
      ---         BLOCKEND  ---      ---       LVL=0

      01000A7BH   BLOCK     CODE     ---       LVL=0
      00000003H   SYMBOL    DATA     CHAR      c
      01000A7BH   LINE      CODE     ---       #185
      01000A7DH   LINE      CODE     ---       #186
      01000A7DH   LINE      CODE     ---       #187
      ---         BLOCKEND  ---      ---       LVL=0

      ---         MODULE    ---      ---       LVD
      02000079H   PUBLIC    XDATA    BYTE      lvd_flag
      01000A5EH   PUBLIC    CODE     ---       lvd_init
      01000003H   PUBLIC    CODE     ---       EFC_IRQHandler
      00000098H.3 SFRSYM    DATA     BIT       TB80
      000000E0H.7 SFRSYM    DATA     BIT       ACC7
      00000080H   SFRSYM    DATA     BYTE      P0
      00000090H   SFRSYM    DATA     BYTE      P1
      000000A0H   SFRSYM    DATA     BYTE      P2
      00000098H.5 SFRSYM    DATA     BIT       SM20
      000000B2H   SFRSYM    DATA     BYTE      ESTCR
      000000B1H   SFRSYM    DATA     BYTE      CLKST
      000000D0H.6 SFRSYM    DATA     BIT       AC
      000000D8H.3 SFRSYM    DATA     BIT       ERSTF
      000000E6H   SFRSYM    DATA     BYTE      PRESET0
      000000D4H   SFRSYM    DATA     BYTE      OCTRL
      000000A8H.7 SFRSYM    DATA     BIT       EA
      0000008FH   SFRSYM    DATA     BYTE      POREN
      000000C8H   SFRSYM    DATA     BYTE      PWM0CON
      000000E7H   SFRSYM    DATA     BYTE      PRESET1
      000000C9H   SFRSYM    DATA     BYTE      PWM1CON
      00000086H   SFRSYM    DATA     BYTE      BEEPCTR
      000000CAH   SFRSYM    DATA     BYTE      PWM2CON
      000000B8H.4 SFRSYM    DATA     BIT       LPTIMINTEN
      000000ABH   SFRSYM    DATA     BYTE      P0AH
      000000B0H   SFRSYM    DATA     BYTE      P1AH
      000000E8H   SFRSYM    DATA     BYTE      P2AH
      000000F8H.6 SFRSYM    DATA     BIT       RC32KF
      000000A8H   SFRSYM    DATA     BYTE      IEN0
      000000A7H   SFRSYM    DATA     BYTE      OPSET
      000000A4H   SFRSYM    DATA     BYTE      P0AL
      000000B8H   SFRSYM    DATA     BYTE      IEN1
      000000A8H.6 SFRSYM    DATA     BIT       EADC
      00000085H   SFRSYM    DATA     BYTE      DPH1
      000000AEH   SFRSYM    DATA     BYTE      P1AL
      0000009AH   SFRSYM    DATA     BYTE      IEN2
      000000C0H   SFRSYM    DATA     BYTE      P2AL
      000000B6H   SFRSYM    DATA     BYTE      ADCDR0
      000000F8H.5 SFRSYM    DATA     BIT       RC16MF
      000000B7H   SFRSYM    DATA     BYTE      ADCDR1
LX51 LINKER/LOCATER V4.66.97.0                                                        07/19/2022  10:30:28  PAGE 22


      00000084H   SFRSYM    DATA     BYTE      DPL1
      000000D6H   SFRSYM    DATA     BYTE      P0OD
      000000DBH   SFRSYM    DATA     BYTE      P1OD
      000000D5H   SFRSYM    DATA     BYTE      P0PD
      00000098H.4 SFRSYM    DATA     BIT       REN0
      000000ECH   SFRSYM    DATA     BYTE      P2OD
      000000DAH   SFRSYM    DATA     BYTE      P1PD
      000000E4H   SFRSYM    DATA     BYTE      P2PD
      000000D7H   SFRSYM    DATA     BYTE      P0CS
      00000097H   SFRSYM    DATA     BYTE      P0DR
      0000009EH   SFRSYM    DATA     BYTE      EUARTEN
      000000DCH   SFRSYM    DATA     BYTE      P1CS
      000000E5H   SFRSYM    DATA     BYTE      P1DR
      000000F4H   SFRSYM    DATA     BYTE      P2CS
      000000FCH   SFRSYM    DATA     BYTE      P2DR
      000000D0H.7 SFRSYM    DATA     BIT       CY
      000000D8H.0 SFRSYM    DATA     BIT       WDT0
      000000D8H.1 SFRSYM    DATA     BIT       WDT1
      000000D8H.2 SFRSYM    DATA     BIT       WDT2
      00000081H   SFRSYM    DATA     BYTE      SP
      000000F1H   SFRSYM    DATA     BYTE      P0PU
      000000F2H   SFRSYM    DATA     BYTE      P1PU
      000000D1H   SFRSYM    DATA     WORD      OADR
      000000F3H   SFRSYM    DATA     BYTE      P2PU
      00000093H   SFRSYM    DATA     BYTE      ADCIER
      000000A5H   SFRSYM    DATA     BYTE      OSEC
      000000D8H.6 SFRSYM    DATA     BIT       WDEN
      000000BAH   SFRSYM    DATA     BYTE      S0RELH
      00000080H.0 SFRSYM    DATA     BIT       P00
      000000D8H.7 SFRSYM    DATA     BIT       WDOF
      000000BBH   SFRSYM    DATA     BYTE      S1RELH
      00000090H.0 SFRSYM    DATA     BIT       P10
      00000080H.1 SFRSYM    DATA     BIT       P01
      00000087H   SFRSYM    DATA     BYTE      PCON
      000000C4H   SFRSYM    DATA     BYTE      PWM0DH
      000000A0H.0 SFRSYM    DATA     BIT       P20
      00000090H.1 SFRSYM    DATA     BIT       P11
      00000080H.2 SFRSYM    DATA     BIT       P02
      000000C6H   SFRSYM    DATA     BYTE      PWM1DH
      00000090H.2 SFRSYM    DATA     BIT       P12
      00000080H.3 SFRSYM    DATA     BIT       P03
      000000C7H   SFRSYM    DATA     BYTE      PWM2DH
      000000C8H.2 SFRSYM    DATA     BIT       PWM0IE
      000000AAH   SFRSYM    DATA     BYTE      S0RELL
      000000A0H.2 SFRSYM    DATA     BIT       P22
      00000090H.3 SFRSYM    DATA     BIT       P13
      00000080H.4 SFRSYM    DATA     BIT       P04
      000000C8H.1 SFRSYM    DATA     BIT       PWM0IF
      0000009DH   SFRSYM    DATA     BYTE      S1RELL
      000000A0H.3 SFRSYM    DATA     BIT       P23
      00000090H.4 SFRSYM    DATA     BIT       P14
      00000080H.5 SFRSYM    DATA     BIT       P05
      000000C3H   SFRSYM    DATA     BYTE      PWM0DL
      00000090H.5 SFRSYM    DATA     BIT       P15
      000000A6H   SFRSYM    DATA     BYTE      OSTATUS
      000000C5H   SFRSYM    DATA     BYTE      PWM1DL
      000000A0H.5 SFRSYM    DATA     BIT       P25
      000000D8H.4 SFRSYM    DATA     BIT       PORF
      000000D8H   SFRSYM    DATA     BYTE      RSTSTAT
      000000CFH   SFRSYM    DATA     BYTE      PWM2DL
      000000A0H.6 SFRSYM    DATA     BIT       P26
      000000C8H.7 SFRSYM    DATA     BIT       PWM0EN
      000000A0H.7 SFRSYM    DATA     BIT       P27
      000000A8H.5 SFRSYM    DATA     BIT       EPWM
      000000D8H.5 SFRSYM    DATA     BIT       LVRF
LX51 LINKER/LOCATER V4.66.97.0                                                        07/19/2022  10:30:28  PAGE 23


      000000F8H   SFRSYM    DATA     BYTE      CLKCON
      000000CCH   SFRSYM    DATA     BYTE      PWM0PH
      000000CEH   SFRSYM    DATA     BYTE      PWM1PH
      000000B8H.5 SFRSYM    DATA     BIT       I2CINTEN
      000000C2H   SFRSYM    DATA     BYTE      PWM2PH
      000000F0H   SFRSYM    DATA     BYTE      B
      000000EEH   SFRSYM    DATA     BYTE      RCHDIV
      000000CBH   SFRSYM    DATA     BYTE      PWM0PL
      000000CDH   SFRSYM    DATA     BYTE      PWM1PL
      000000C1H   SFRSYM    DATA     BYTE      PWM2PL
      000000F7H   SFRSYM    DATA     BYTE      ADCSPW
      000000F8H.1 SFRSYM    DATA     BIT       XCLKEN
      000000E0H   SFRSYM    DATA     BYTE      ACC
      000000DDH   SFRSYM    DATA     BYTE      LVDCON
      000000A8H.4 SFRSYM    DATA     BIT       ES0
      000000A9H   SFRSYM    DATA     BYTE      IP0
      000000A8H.1 SFRSYM    DATA     BIT       ET0
      000000A8H.2 SFRSYM    DATA     BIT       ES1
      000000F6H   SFRSYM    DATA     BYTE      ADCCSTAT
      000000B9H   SFRSYM    DATA     BYTE      IP1
      000000A8H.3 SFRSYM    DATA     BIT       ET1
      00000098H.0 SFRSYM    DATA     BIT       RI0
      000000C8H.0 SFRSYM    DATA     BIT       PWM0SS
      00000098H.1 SFRSYM    DATA     BIT       TI0
      000000A8H.0 SFRSYM    DATA     BIT       EX0
      000000D0H.0 SFRSYM    DATA     BIT       P
      000000B8H.3 SFRSYM    DATA     BIT       EFCINTEN
      000000A2H   SFRSYM    DATA     BYTE      OINTEN
      00000098H.7 SFRSYM    DATA     BIT       SM0
      00000098H.6 SFRSYM    DATA     BIT       SM1
      000000FEH   SFRSYM    DATA     BYTE      ADCCDR0
      000000FFH   SFRSYM    DATA     BYTE      ADCCDR1
      000000D0H.3 SFRSYM    DATA     BIT       RS0
      000000ACH   SFRSYM    DATA     BYTE      ADCGCR0
      000000D0H.4 SFRSYM    DATA     BIT       RS1
      000000ADH   SFRSYM    DATA     BYTE      ADCGCR1
      000000B4H   SFRSYM    DATA     BYTE      ADCGCR2
      000000B5H   SFRSYM    DATA     BYTE      ADCGCR3
      000000F8H.3 SFRSYM    DATA     BIT       RC32KEN
      000000DEH   SFRSYM    DATA     BYTE      PCLK0
      000000DFH   SFRSYM    DATA     BYTE      PCLK1
      00000083H   SFRSYM    DATA     BYTE      DPH
      000000E9H   SFRSYM    DATA     BYTE      P0IEN
      000000F5H   SFRSYM    DATA     BYTE      ADCHL
      000000F8H.2 SFRSYM    DATA     BIT       RC16MEN
      000000EAH   SFRSYM    DATA     BYTE      P1IEN
      000000EBH   SFRSYM    DATA     BYTE      P2IEN
      000000B6H   SFRSYM    DATA     WORD      ADCDR
      000000B3H   SFRSYM    DATA     BYTE      XTHCTR
      00000082H   SFRSYM    DATA     BYTE      DPL
      00000099H   SFRSYM    DATA     BYTE      S0BUF
      0000009CH   SFRSYM    DATA     BYTE      S1BUF
      000000F9H   SFRSYM    DATA     BYTE      P0OEN
      000000B8H.0 SFRSYM    DATA     BIT       GTIM0INTEN
      000000D9H   SFRSYM    DATA     BYTE      SYSDIV
      00000098H   SFRSYM    DATA     BYTE      S0CON
      000000FAH   SFRSYM    DATA     BYTE      P1OEN
      000000B8H.2 SFRSYM    DATA     BIT       GTIM1INTEN
      000000A3H   SFRSYM    DATA     BYTE      OINTUS
      000000BEH   SFRSYM    DATA     BYTE      RCHTRIMH
      000000F8H.0 SFRSYM    DATA     BIT       SYSSEL
      0000009BH   SFRSYM    DATA     BYTE      S1CON
      000000FBH   SFRSYM    DATA     BYTE      P2OEN
      000000B8H.6 SFRSYM    DATA     BIT       GTIM2INTEN
      000000BDH   SFRSYM    DATA     BYTE      LDOTRIMH
LX51 LINKER/LOCATER V4.66.97.0                                                        07/19/2022  10:30:28  PAGE 24


      00000092H   SFRSYM    DATA     BYTE      DPS
      0000009FH   SFRSYM    DATA     BYTE      RCLTRIMH
      000000BFH   SFRSYM    DATA     BYTE      RCHTRIML
      000000D3H   SFRSYM    DATA     BYTE      ODATA
      00000091H   SFRSYM    DATA     BYTE      LDOTRIML
      000000BCH   SFRSYM    DATA     BYTE      RCLTRIML
      000000E1H   SFRSYM    DATA     BYTE      P0IRQ
      000000B8H.1 SFRSYM    DATA     BIT       SPIINTEN
      000000E2H   SFRSYM    DATA     BYTE      P1IRQ
      000000E3H   SFRSYM    DATA     BYTE      P2IRQ
      000000D2H   SFRSYM    DATA     BYTE      OADRH
      000000B8H.7 SFRSYM    DATA     BIT       UART2INTEN
      000000F0H.0 SFRSYM    DATA     BIT       B0
      000000F0H.1 SFRSYM    DATA     BIT       B1
      000000F0H.2 SFRSYM    DATA     BIT       B2
      000000D1H   SFRSYM    DATA     BYTE      OADRL
      000000F0H.3 SFRSYM    DATA     BIT       B3
      000000F0H.4 SFRSYM    DATA     BIT       B4
      000000D0H.5 SFRSYM    DATA     BIT       F0
      000000F0H.5 SFRSYM    DATA     BIT       B5
      000000D0H.1 SFRSYM    DATA     BIT       F1
      000000AFH   SFRSYM    DATA     BYTE      REMAP
      000000F0H.6 SFRSYM    DATA     BIT       B6
      000000E0H.0 SFRSYM    DATA     BIT       ACC0
      000000A1H   SFRSYM    DATA     BYTE      OUS
      000000C8H.6 SFRSYM    DATA     BIT       PWM0S
      000000F0H.7 SFRSYM    DATA     BIT       B7
      000000E0H.1 SFRSYM    DATA     BIT       ACC1
      000000F8H.4 SFRSYM    DATA     BIT       XCLKF
      000000E0H.2 SFRSYM    DATA     BIT       ACC2
      0000008EH   SFRSYM    DATA     BYTE      PDSEL
      000000E0H.3 SFRSYM    DATA     BIT       ACC3
      000000D0H   SFRSYM    DATA     BYTE      PSW
      000000E0H.4 SFRSYM    DATA     BIT       ACC4
      00000098H.2 SFRSYM    DATA     BIT       RB80
      000000E0H.5 SFRSYM    DATA     BIT       ACC5
      000000FDH   SFRSYM    DATA     BYTE      ADCVREF
      000000E0H.6 SFRSYM    DATA     BIT       ACC6

      01000003H   BLOCK     CODE     ---       LVL=0
      01000003H   LINE      CODE     ---       #5
      01000009H   LINE      CODE     ---       #7
      0100000EH   LINE      CODE     ---       #8
      0100000EH   LINE      CODE     ---       #9
      01000014H   LINE      CODE     ---       #10
      01000017H   LINE      CODE     ---       #11
      01000017H   LINE      CODE     ---       #13
      0100001AH   LINE      CODE     ---       #15
      ---         BLOCKEND  ---      ---       LVL=0

      01000A5EH   BLOCK     CODE     ---       LVL=0
      01000A5EH   LINE      CODE     ---       #19
      01000A5EH   LINE      CODE     ---       #20
      01000A5EH   LINE      CODE     ---       #21
      01000A61H   LINE      CODE     ---       #22
      01000A64H   LINE      CODE     ---       #23
      01000A67H   LINE      CODE     ---       #24
      01000A6AH   LINE      CODE     ---       #25
      01000A6DH   LINE      CODE     ---       #27
      01000A6FH   LINE      CODE     ---       #29
      ---         BLOCKEND  ---      ---       LVL=0

      ---         MODULE    ---      ---       APP
      02000043H   PUBLIC    XDATA    WORD      tx_count
      02000041H   PUBLIC    XDATA    WORD      rx_count
LX51 LINKER/LOCATER V4.66.97.0                                                        07/19/2022  10:30:28  PAGE 25


      02000040H   PUBLIC    XDATA    BYTE      rx_flag
      02000020H   PUBLIC    XDATA    ---       uart0_tx_buf
      02000000H   PUBLIC    XDATA    ---       uart0_rx_buf
      0100098BH   PUBLIC    CODE     ---       lvd_test
      01000A1DH   PUBLIC    CODE     ---       uart_init
      010009FBH   PUBLIC    CODE     ---       uart0_rec_pro
      00000098H.3 SFRSYM    DATA     BIT       TB80
      000000E0H.7 SFRSYM    DATA     BIT       ACC7
      00000080H   SFRSYM    DATA     BYTE      P0
      00000090H   SFRSYM    DATA     BYTE      P1
      000000A0H   SFRSYM    DATA     BYTE      P2
      00000098H.5 SFRSYM    DATA     BIT       SM20
      000000B2H   SFRSYM    DATA     BYTE      ESTCR
      000000B1H   SFRSYM    DATA     BYTE      CLKST
      000000D0H.6 SFRSYM    DATA     BIT       AC
      000000D8H.3 SFRSYM    DATA     BIT       ERSTF
      000000E6H   SFRSYM    DATA     BYTE      PRESET0
      000000D4H   SFRSYM    DATA     BYTE      OCTRL
      000000A8H.7 SFRSYM    DATA     BIT       EA
      0000008FH   SFRSYM    DATA     BYTE      POREN
      000000C8H   SFRSYM    DATA     BYTE      PWM0CON
      000000E7H   SFRSYM    DATA     BYTE      PRESET1
      000000C9H   SFRSYM    DATA     BYTE      PWM1CON
      00000086H   SFRSYM    DATA     BYTE      BEEPCTR
      000000CAH   SFRSYM    DATA     BYTE      PWM2CON
      000000B8H.4 SFRSYM    DATA     BIT       LPTIMINTEN
      000000ABH   SFRSYM    DATA     BYTE      P0AH
      000000B0H   SFRSYM    DATA     BYTE      P1AH
      000000E8H   SFRSYM    DATA     BYTE      P2AH
      000000F8H.6 SFRSYM    DATA     BIT       RC32KF
      000000A8H   SFRSYM    DATA     BYTE      IEN0
      000000A7H   SFRSYM    DATA     BYTE      OPSET
      000000A4H   SFRSYM    DATA     BYTE      P0AL
      000000B8H   SFRSYM    DATA     BYTE      IEN1
      000000A8H.6 SFRSYM    DATA     BIT       EADC
      00000085H   SFRSYM    DATA     BYTE      DPH1
      000000AEH   SFRSYM    DATA     BYTE      P1AL
      0000009AH   SFRSYM    DATA     BYTE      IEN2
      000000C0H   SFRSYM    DATA     BYTE      P2AL
      000000B6H   SFRSYM    DATA     BYTE      ADCDR0
      000000F8H.5 SFRSYM    DATA     BIT       RC16MF
      000000B7H   SFRSYM    DATA     BYTE      ADCDR1
      00000084H   SFRSYM    DATA     BYTE      DPL1
      000000D6H   SFRSYM    DATA     BYTE      P0OD
      000000DBH   SFRSYM    DATA     BYTE      P1OD
      000000D5H   SFRSYM    DATA     BYTE      P0PD
      00000098H.4 SFRSYM    DATA     BIT       REN0
      000000ECH   SFRSYM    DATA     BYTE      P2OD
      000000DAH   SFRSYM    DATA     BYTE      P1PD
      000000E4H   SFRSYM    DATA     BYTE      P2PD
      000000D7H   SFRSYM    DATA     BYTE      P0CS
      00000097H   SFRSYM    DATA     BYTE      P0DR
      0000009EH   SFRSYM    DATA     BYTE      EUARTEN
      000000DCH   SFRSYM    DATA     BYTE      P1CS
      000000E5H   SFRSYM    DATA     BYTE      P1DR
      000000F4H   SFRSYM    DATA     BYTE      P2CS
      000000FCH   SFRSYM    DATA     BYTE      P2DR
      000000D0H.7 SFRSYM    DATA     BIT       CY
      000000D8H.0 SFRSYM    DATA     BIT       WDT0
      000000D8H.1 SFRSYM    DATA     BIT       WDT1
      000000D8H.2 SFRSYM    DATA     BIT       WDT2
      00000081H   SFRSYM    DATA     BYTE      SP
      000000F1H   SFRSYM    DATA     BYTE      P0PU
      000000F2H   SFRSYM    DATA     BYTE      P1PU
      000000D1H   SFRSYM    DATA     WORD      OADR
LX51 LINKER/LOCATER V4.66.97.0                                                        07/19/2022  10:30:28  PAGE 26


      000000F3H   SFRSYM    DATA     BYTE      P2PU
      00000093H   SFRSYM    DATA     BYTE      ADCIER
      000000A5H   SFRSYM    DATA     BYTE      OSEC
      000000D8H.6 SFRSYM    DATA     BIT       WDEN
      000000BAH   SFRSYM    DATA     BYTE      S0RELH
      00000080H.0 SFRSYM    DATA     BIT       P00
      000000D8H.7 SFRSYM    DATA     BIT       WDOF
      000000BBH   SFRSYM    DATA     BYTE      S1RELH
      00000090H.0 SFRSYM    DATA     BIT       P10
      00000080H.1 SFRSYM    DATA     BIT       P01
      00000087H   SFRSYM    DATA     BYTE      PCON
      000000C4H   SFRSYM    DATA     BYTE      PWM0DH
      000000A0H.0 SFRSYM    DATA     BIT       P20
      00000090H.1 SFRSYM    DATA     BIT       P11
      00000080H.2 SFRSYM    DATA     BIT       P02
      000000C6H   SFRSYM    DATA     BYTE      PWM1DH
      00000090H.2 SFRSYM    DATA     BIT       P12
      00000080H.3 SFRSYM    DATA     BIT       P03
      000000C7H   SFRSYM    DATA     BYTE      PWM2DH
      000000C8H.2 SFRSYM    DATA     BIT       PWM0IE
      000000AAH   SFRSYM    DATA     BYTE      S0RELL
      000000A0H.2 SFRSYM    DATA     BIT       P22
      00000090H.3 SFRSYM    DATA     BIT       P13
      00000080H.4 SFRSYM    DATA     BIT       P04
      000000C8H.1 SFRSYM    DATA     BIT       PWM0IF
      0000009DH   SFRSYM    DATA     BYTE      S1RELL
      000000A0H.3 SFRSYM    DATA     BIT       P23
      00000090H.4 SFRSYM    DATA     BIT       P14
      00000080H.5 SFRSYM    DATA     BIT       P05
      000000C3H   SFRSYM    DATA     BYTE      PWM0DL
      00000090H.5 SFRSYM    DATA     BIT       P15
      000000A6H   SFRSYM    DATA     BYTE      OSTATUS
      000000C5H   SFRSYM    DATA     BYTE      PWM1DL
      000000A0H.5 SFRSYM    DATA     BIT       P25
      000000D8H.4 SFRSYM    DATA     BIT       PORF
      000000D8H   SFRSYM    DATA     BYTE      RSTSTAT
      000000CFH   SFRSYM    DATA     BYTE      PWM2DL
      000000A0H.6 SFRSYM    DATA     BIT       P26
      000000C8H.7 SFRSYM    DATA     BIT       PWM0EN
      000000A0H.7 SFRSYM    DATA     BIT       P27
      000000A8H.5 SFRSYM    DATA     BIT       EPWM
      000000D8H.5 SFRSYM    DATA     BIT       LVRF
      000000F8H   SFRSYM    DATA     BYTE      CLKCON
      000000CCH   SFRSYM    DATA     BYTE      PWM0PH
      000000CEH   SFRSYM    DATA     BYTE      PWM1PH
      000000B8H.5 SFRSYM    DATA     BIT       I2CINTEN
      000000C2H   SFRSYM    DATA     BYTE      PWM2PH
      000000F0H   SFRSYM    DATA     BYTE      B
      000000EEH   SFRSYM    DATA     BYTE      RCHDIV
      000000CBH   SFRSYM    DATA     BYTE      PWM0PL
      000000CDH   SFRSYM    DATA     BYTE      PWM1PL
      000000C1H   SFRSYM    DATA     BYTE      PWM2PL
      000000F7H   SFRSYM    DATA     BYTE      ADCSPW
      000000F8H.1 SFRSYM    DATA     BIT       XCLKEN
      000000E0H   SFRSYM    DATA     BYTE      ACC
      000000DDH   SFRSYM    DATA     BYTE      LVDCON
      000000A8H.4 SFRSYM    DATA     BIT       ES0
      000000A9H   SFRSYM    DATA     BYTE      IP0
      000000A8H.1 SFRSYM    DATA     BIT       ET0
      000000A8H.2 SFRSYM    DATA     BIT       ES1
      000000F6H   SFRSYM    DATA     BYTE      ADCCSTAT
      000000B9H   SFRSYM    DATA     BYTE      IP1
      000000A8H.3 SFRSYM    DATA     BIT       ET1
      00000098H.0 SFRSYM    DATA     BIT       RI0
      000000C8H.0 SFRSYM    DATA     BIT       PWM0SS
LX51 LINKER/LOCATER V4.66.97.0                                                        07/19/2022  10:30:28  PAGE 27


      00000098H.1 SFRSYM    DATA     BIT       TI0
      000000A8H.0 SFRSYM    DATA     BIT       EX0
      000000D0H.0 SFRSYM    DATA     BIT       P
      000000B8H.3 SFRSYM    DATA     BIT       EFCINTEN
      000000A2H   SFRSYM    DATA     BYTE      OINTEN
      00000098H.7 SFRSYM    DATA     BIT       SM0
      00000098H.6 SFRSYM    DATA     BIT       SM1
      000000FEH   SFRSYM    DATA     BYTE      ADCCDR0
      000000FFH   SFRSYM    DATA     BYTE      ADCCDR1
      000000D0H.3 SFRSYM    DATA     BIT       RS0
      000000ACH   SFRSYM    DATA     BYTE      ADCGCR0
      000000D0H.4 SFRSYM    DATA     BIT       RS1
      000000ADH   SFRSYM    DATA     BYTE      ADCGCR1
      000000B4H   SFRSYM    DATA     BYTE      ADCGCR2
      000000B5H   SFRSYM    DATA     BYTE      ADCGCR3
      000000F8H.3 SFRSYM    DATA     BIT       RC32KEN
      000000DEH   SFRSYM    DATA     BYTE      PCLK0
      000000DFH   SFRSYM    DATA     BYTE      PCLK1
      00000083H   SFRSYM    DATA     BYTE      DPH
      000000E9H   SFRSYM    DATA     BYTE      P0IEN
      000000F5H   SFRSYM    DATA     BYTE      ADCHL
      000000F8H.2 SFRSYM    DATA     BIT       RC16MEN
      000000EAH   SFRSYM    DATA     BYTE      P1IEN
      000000EBH   SFRSYM    DATA     BYTE      P2IEN
      000000B6H   SFRSYM    DATA     WORD      ADCDR
      000000B3H   SFRSYM    DATA     BYTE      XTHCTR
      00000082H   SFRSYM    DATA     BYTE      DPL
      00000099H   SFRSYM    DATA     BYTE      S0BUF
      0000009CH   SFRSYM    DATA     BYTE      S1BUF
      000000F9H   SFRSYM    DATA     BYTE      P0OEN
      000000B8H.0 SFRSYM    DATA     BIT       GTIM0INTEN
      000000D9H   SFRSYM    DATA     BYTE      SYSDIV
      00000098H   SFRSYM    DATA     BYTE      S0CON
      000000FAH   SFRSYM    DATA     BYTE      P1OEN
      000000B8H.2 SFRSYM    DATA     BIT       GTIM1INTEN
      000000A3H   SFRSYM    DATA     BYTE      OINTUS
      000000BEH   SFRSYM    DATA     BYTE      RCHTRIMH
      000000F8H.0 SFRSYM    DATA     BIT       SYSSEL
      0000009BH   SFRSYM    DATA     BYTE      S1CON
      000000FBH   SFRSYM    DATA     BYTE      P2OEN
      000000B8H.6 SFRSYM    DATA     BIT       GTIM2INTEN
      000000BDH   SFRSYM    DATA     BYTE      LDOTRIMH
      00000092H   SFRSYM    DATA     BYTE      DPS
      0000009FH   SFRSYM    DATA     BYTE      RCLTRIMH
      000000BFH   SFRSYM    DATA     BYTE      RCHTRIML
      000000D3H   SFRSYM    DATA     BYTE      ODATA
      00000091H   SFRSYM    DATA     BYTE      LDOTRIML
      000000BCH   SFRSYM    DATA     BYTE      RCLTRIML
      000000E1H   SFRSYM    DATA     BYTE      P0IRQ
      000000B8H.1 SFRSYM    DATA     BIT       SPIINTEN
      000000E2H   SFRSYM    DATA     BYTE      P1IRQ
      000000E3H   SFRSYM    DATA     BYTE      P2IRQ
      000000D2H   SFRSYM    DATA     BYTE      OADRH
      000000B8H.7 SFRSYM    DATA     BIT       UART2INTEN
      000000F0H.0 SFRSYM    DATA     BIT       B0
      000000F0H.1 SFRSYM    DATA     BIT       B1
      000000F0H.2 SFRSYM    DATA     BIT       B2
      000000D1H   SFRSYM    DATA     BYTE      OADRL
      000000F0H.3 SFRSYM    DATA     BIT       B3
      000000F0H.4 SFRSYM    DATA     BIT       B4
      000000D0H.5 SFRSYM    DATA     BIT       F0
      000000F0H.5 SFRSYM    DATA     BIT       B5
      000000D0H.1 SFRSYM    DATA     BIT       F1
      000000AFH   SFRSYM    DATA     BYTE      REMAP
      000000F0H.6 SFRSYM    DATA     BIT       B6
LX51 LINKER/LOCATER V4.66.97.0                                                        07/19/2022  10:30:28  PAGE 28


      000000E0H.0 SFRSYM    DATA     BIT       ACC0
      000000A1H   SFRSYM    DATA     BYTE      OUS
      000000C8H.6 SFRSYM    DATA     BIT       PWM0S
      000000F0H.7 SFRSYM    DATA     BIT       B7
      000000E0H.1 SFRSYM    DATA     BIT       ACC1
      000000F8H.4 SFRSYM    DATA     BIT       XCLKF
      000000E0H.2 SFRSYM    DATA     BIT       ACC2
      0000008EH   SFRSYM    DATA     BYTE      PDSEL
      000000E0H.3 SFRSYM    DATA     BIT       ACC3
      000000D0H   SFRSYM    DATA     BYTE      PSW
      000000E0H.4 SFRSYM    DATA     BIT       ACC4
      00000098H.2 SFRSYM    DATA     BIT       RB80
      000000E0H.5 SFRSYM    DATA     BIT       ACC5
      000000FDH   SFRSYM    DATA     BYTE      ADCVREF
      000000E0H.6 SFRSYM    DATA     BIT       ACC6

      010009FBH   BLOCK     CODE     ---       LVL=0
      010009FBH   LINE      CODE     ---       #30
      010009FBH   LINE      CODE     ---       #31
      010009FBH   LINE      CODE     ---       #32
      01000A16H   LINE      CODE     ---       #33
      01000A1CH   LINE      CODE     ---       #34
      ---         BLOCKEND  ---      ---       LVL=0

      01000A1DH   BLOCK     CODE     ---       LVL=0
      01000A1DH   LINE      CODE     ---       #43
      01000A1DH   LINE      CODE     ---       #44
      01000A1DH   LINE      CODE     ---       #45
      01000A22H   LINE      CODE     ---       #46
      01000A2BH   LINE      CODE     ---       #47
      ---         BLOCKEND  ---      ---       LVL=0

      0100098BH   BLOCK     CODE     ---       LVL=0
      0100098BH   LINE      CODE     ---       #57
      0100098BH   LINE      CODE     ---       #58
      0100098BH   LINE      CODE     ---       #59
      010009A0H   LINE      CODE     ---       #60
      010009A9H   LINE      CODE     ---       #62
      010009ACH   LINE      CODE     ---       #64
      010009ACH   LINE      CODE     ---       #65
      010009ACH   LINE      CODE     ---       #66
      010009B4H   LINE      CODE     ---       #67
      010009B4H   LINE      CODE     ---       #68
      010009BDH   LINE      CODE     ---       #69
      010009C2H   LINE      CODE     ---       #70
      010009C2H   LINE      CODE     ---       #71
      ---         BLOCKEND  ---      ---       LVL=0

      ---         MODULE    ---      ---       MAIN
      01000A70H   PUBLIC    CODE     ---       main
      00000098H.3 SFRSYM    DATA     BIT       TB80
      000000E0H.7 SFRSYM    DATA     BIT       ACC7
      00000080H   SFRSYM    DATA     BYTE      P0
      00000090H   SFRSYM    DATA     BYTE      P1
      000000A0H   SFRSYM    DATA     BYTE      P2
      00000098H.5 SFRSYM    DATA     BIT       SM20
      000000B2H   SFRSYM    DATA     BYTE      ESTCR
      000000B1H   SFRSYM    DATA     BYTE      CLKST
      000000D0H.6 SFRSYM    DATA     BIT       AC
      000000D8H.3 SFRSYM    DATA     BIT       ERSTF
      000000E6H   SFRSYM    DATA     BYTE      PRESET0
      000000D4H   SFRSYM    DATA     BYTE      OCTRL
      000000A8H.7 SFRSYM    DATA     BIT       EA
      0000008FH   SFRSYM    DATA     BYTE      POREN
      000000C8H   SFRSYM    DATA     BYTE      PWM0CON
LX51 LINKER/LOCATER V4.66.97.0                                                        07/19/2022  10:30:28  PAGE 29


      000000E7H   SFRSYM    DATA     BYTE      PRESET1
      000000C9H   SFRSYM    DATA     BYTE      PWM1CON
      00000086H   SFRSYM    DATA     BYTE      BEEPCTR
      000000CAH   SFRSYM    DATA     BYTE      PWM2CON
      000000B8H.4 SFRSYM    DATA     BIT       LPTIMINTEN
      000000ABH   SFRSYM    DATA     BYTE      P0AH
      000000B0H   SFRSYM    DATA     BYTE      P1AH
      000000E8H   SFRSYM    DATA     BYTE      P2AH
      000000F8H.6 SFRSYM    DATA     BIT       RC32KF
      000000A8H   SFRSYM    DATA     BYTE      IEN0
      000000A7H   SFRSYM    DATA     BYTE      OPSET
      000000A4H   SFRSYM    DATA     BYTE      P0AL
      000000B8H   SFRSYM    DATA     BYTE      IEN1
      000000A8H.6 SFRSYM    DATA     BIT       EADC
      00000085H   SFRSYM    DATA     BYTE      DPH1
      000000AEH   SFRSYM    DATA     BYTE      P1AL
      0000009AH   SFRSYM    DATA     BYTE      IEN2
      000000C0H   SFRSYM    DATA     BYTE      P2AL
      000000B6H   SFRSYM    DATA     BYTE      ADCDR0
      000000F8H.5 SFRSYM    DATA     BIT       RC16MF
      000000B7H   SFRSYM    DATA     BYTE      ADCDR1
      00000084H   SFRSYM    DATA     BYTE      DPL1
      000000D6H   SFRSYM    DATA     BYTE      P0OD
      000000DBH   SFRSYM    DATA     BYTE      P1OD
      000000D5H   SFRSYM    DATA     BYTE      P0PD
      00000098H.4 SFRSYM    DATA     BIT       REN0
      000000ECH   SFRSYM    DATA     BYTE      P2OD
      000000DAH   SFRSYM    DATA     BYTE      P1PD
      000000E4H   SFRSYM    DATA     BYTE      P2PD
      000000D7H   SFRSYM    DATA     BYTE      P0CS
      00000097H   SFRSYM    DATA     BYTE      P0DR
      0000009EH   SFRSYM    DATA     BYTE      EUARTEN
      000000DCH   SFRSYM    DATA     BYTE      P1CS
      000000E5H   SFRSYM    DATA     BYTE      P1DR
      000000F4H   SFRSYM    DATA     BYTE      P2CS
      000000FCH   SFRSYM    DATA     BYTE      P2DR
      000000D0H.7 SFRSYM    DATA     BIT       CY
      000000D8H.0 SFRSYM    DATA     BIT       WDT0
      000000D8H.1 SFRSYM    DATA     BIT       WDT1
      000000D8H.2 SFRSYM    DATA     BIT       WDT2
      00000081H   SFRSYM    DATA     BYTE      SP
      000000F1H   SFRSYM    DATA     BYTE      P0PU
      000000F2H   SFRSYM    DATA     BYTE      P1PU
      000000D1H   SFRSYM    DATA     WORD      OADR
      000000F3H   SFRSYM    DATA     BYTE      P2PU
      00000093H   SFRSYM    DATA     BYTE      ADCIER
      000000A5H   SFRSYM    DATA     BYTE      OSEC
      000000D8H.6 SFRSYM    DATA     BIT       WDEN
      000000BAH   SFRSYM    DATA     BYTE      S0RELH
      00000080H.0 SFRSYM    DATA     BIT       P00
      000000D8H.7 SFRSYM    DATA     BIT       WDOF
      000000BBH   SFRSYM    DATA     BYTE      S1RELH
      00000090H.0 SFRSYM    DATA     BIT       P10
      00000080H.1 SFRSYM    DATA     BIT       P01
      00000087H   SFRSYM    DATA     BYTE      PCON
      000000C4H   SFRSYM    DATA     BYTE      PWM0DH
      000000A0H.0 SFRSYM    DATA     BIT       P20
      00000090H.1 SFRSYM    DATA     BIT       P11
      00000080H.2 SFRSYM    DATA     BIT       P02
      000000C6H   SFRSYM    DATA     BYTE      PWM1DH
      00000090H.2 SFRSYM    DATA     BIT       P12
      00000080H.3 SFRSYM    DATA     BIT       P03
      000000C7H   SFRSYM    DATA     BYTE      PWM2DH
      000000C8H.2 SFRSYM    DATA     BIT       PWM0IE
      000000AAH   SFRSYM    DATA     BYTE      S0RELL
LX51 LINKER/LOCATER V4.66.97.0                                                        07/19/2022  10:30:28  PAGE 30


      000000A0H.2 SFRSYM    DATA     BIT       P22
      00000090H.3 SFRSYM    DATA     BIT       P13
      00000080H.4 SFRSYM    DATA     BIT       P04
      000000C8H.1 SFRSYM    DATA     BIT       PWM0IF
      0000009DH   SFRSYM    DATA     BYTE      S1RELL
      000000A0H.3 SFRSYM    DATA     BIT       P23
      00000090H.4 SFRSYM    DATA     BIT       P14
      00000080H.5 SFRSYM    DATA     BIT       P05
      000000C3H   SFRSYM    DATA     BYTE      PWM0DL
      00000090H.5 SFRSYM    DATA     BIT       P15
      000000A6H   SFRSYM    DATA     BYTE      OSTATUS
      000000C5H   SFRSYM    DATA     BYTE      PWM1DL
      000000A0H.5 SFRSYM    DATA     BIT       P25
      000000D8H.4 SFRSYM    DATA     BIT       PORF
      000000D8H   SFRSYM    DATA     BYTE      RSTSTAT
      000000CFH   SFRSYM    DATA     BYTE      PWM2DL
      000000A0H.6 SFRSYM    DATA     BIT       P26
      000000C8H.7 SFRSYM    DATA     BIT       PWM0EN
      000000A0H.7 SFRSYM    DATA     BIT       P27
      000000A8H.5 SFRSYM    DATA     BIT       EPWM
      000000D8H.5 SFRSYM    DATA     BIT       LVRF
      000000F8H   SFRSYM    DATA     BYTE      CLKCON
      000000CCH   SFRSYM    DATA     BYTE      PWM0PH
      000000CEH   SFRSYM    DATA     BYTE      PWM1PH
      000000B8H.5 SFRSYM    DATA     BIT       I2CINTEN
      000000C2H   SFRSYM    DATA     BYTE      PWM2PH
      000000F0H   SFRSYM    DATA     BYTE      B
      000000EEH   SFRSYM    DATA     BYTE      RCHDIV
      000000CBH   SFRSYM    DATA     BYTE      PWM0PL
      000000CDH   SFRSYM    DATA     BYTE      PWM1PL
      000000C1H   SFRSYM    DATA     BYTE      PWM2PL
      000000F7H   SFRSYM    DATA     BYTE      ADCSPW
      000000F8H.1 SFRSYM    DATA     BIT       XCLKEN
      000000E0H   SFRSYM    DATA     BYTE      ACC
      000000DDH   SFRSYM    DATA     BYTE      LVDCON
      000000A8H.4 SFRSYM    DATA     BIT       ES0
      000000A9H   SFRSYM    DATA     BYTE      IP0
      000000A8H.1 SFRSYM    DATA     BIT       ET0
      000000A8H.2 SFRSYM    DATA     BIT       ES1
      000000F6H   SFRSYM    DATA     BYTE      ADCCSTAT
      000000B9H   SFRSYM    DATA     BYTE      IP1
      000000A8H.3 SFRSYM    DATA     BIT       ET1
      00000098H.0 SFRSYM    DATA     BIT       RI0
      000000C8H.0 SFRSYM    DATA     BIT       PWM0SS
      00000098H.1 SFRSYM    DATA     BIT       TI0
      000000A8H.0 SFRSYM    DATA     BIT       EX0
      000000D0H.0 SFRSYM    DATA     BIT       P
      000000B8H.3 SFRSYM    DATA     BIT       EFCINTEN
      000000A2H   SFRSYM    DATA     BYTE      OINTEN
      00000098H.7 SFRSYM    DATA     BIT       SM0
      00000098H.6 SFRSYM    DATA     BIT       SM1
      000000FEH   SFRSYM    DATA     BYTE      ADCCDR0
      000000FFH   SFRSYM    DATA     BYTE      ADCCDR1
      000000D0H.3 SFRSYM    DATA     BIT       RS0
      000000ACH   SFRSYM    DATA     BYTE      ADCGCR0
      000000D0H.4 SFRSYM    DATA     BIT       RS1
      000000ADH   SFRSYM    DATA     BYTE      ADCGCR1
      000000B4H   SFRSYM    DATA     BYTE      ADCGCR2
      000000B5H   SFRSYM    DATA     BYTE      ADCGCR3
      000000F8H.3 SFRSYM    DATA     BIT       RC32KEN
      000000DEH   SFRSYM    DATA     BYTE      PCLK0
      000000DFH   SFRSYM    DATA     BYTE      PCLK1
      00000083H   SFRSYM    DATA     BYTE      DPH
      000000E9H   SFRSYM    DATA     BYTE      P0IEN
      000000F5H   SFRSYM    DATA     BYTE      ADCHL
LX51 LINKER/LOCATER V4.66.97.0                                                        07/19/2022  10:30:28  PAGE 31


      000000F8H.2 SFRSYM    DATA     BIT       RC16MEN
      000000EAH   SFRSYM    DATA     BYTE      P1IEN
      000000EBH   SFRSYM    DATA     BYTE      P2IEN
      000000B6H   SFRSYM    DATA     WORD      ADCDR
      000000B3H   SFRSYM    DATA     BYTE      XTHCTR
      00000082H   SFRSYM    DATA     BYTE      DPL
      00000099H   SFRSYM    DATA     BYTE      S0BUF
      0000009CH   SFRSYM    DATA     BYTE      S1BUF
      000000F9H   SFRSYM    DATA     BYTE      P0OEN
      000000B8H.0 SFRSYM    DATA     BIT       GTIM0INTEN
      000000D9H   SFRSYM    DATA     BYTE      SYSDIV
      00000098H   SFRSYM    DATA     BYTE      S0CON
      000000FAH   SFRSYM    DATA     BYTE      P1OEN
      000000B8H.2 SFRSYM    DATA     BIT       GTIM1INTEN
      000000A3H   SFRSYM    DATA     BYTE      OINTUS
      000000BEH   SFRSYM    DATA     BYTE      RCHTRIMH
      000000F8H.0 SFRSYM    DATA     BIT       SYSSEL
      0000009BH   SFRSYM    DATA     BYTE      S1CON
      000000FBH   SFRSYM    DATA     BYTE      P2OEN
      000000B8H.6 SFRSYM    DATA     BIT       GTIM2INTEN
      000000BDH   SFRSYM    DATA     BYTE      LDOTRIMH
      00000092H   SFRSYM    DATA     BYTE      DPS
      0000009FH   SFRSYM    DATA     BYTE      RCLTRIMH
      000000BFH   SFRSYM    DATA     BYTE      RCHTRIML
      000000D3H   SFRSYM    DATA     BYTE      ODATA
      00000091H   SFRSYM    DATA     BYTE      LDOTRIML
      000000BCH   SFRSYM    DATA     BYTE      RCLTRIML
      000000E1H   SFRSYM    DATA     BYTE      P0IRQ
      000000B8H.1 SFRSYM    DATA     BIT       SPIINTEN
      000000E2H   SFRSYM    DATA     BYTE      P1IRQ
      000000E3H   SFRSYM    DATA     BYTE      P2IRQ
      000000D2H   SFRSYM    DATA     BYTE      OADRH
      000000B8H.7 SFRSYM    DATA     BIT       UART2INTEN
      000000F0H.0 SFRSYM    DATA     BIT       B0
      000000F0H.1 SFRSYM    DATA     BIT       B1
      000000F0H.2 SFRSYM    DATA     BIT       B2
      000000D1H   SFRSYM    DATA     BYTE      OADRL
      000000F0H.3 SFRSYM    DATA     BIT       B3
      000000F0H.4 SFRSYM    DATA     BIT       B4
      000000D0H.5 SFRSYM    DATA     BIT       F0
      000000F0H.5 SFRSYM    DATA     BIT       B5
      000000D0H.1 SFRSYM    DATA     BIT       F1
      000000AFH   SFRSYM    DATA     BYTE      REMAP
      000000F0H.6 SFRSYM    DATA     BIT       B6
      000000E0H.0 SFRSYM    DATA     BIT       ACC0
      000000A1H   SFRSYM    DATA     BYTE      OUS
      000000C8H.6 SFRSYM    DATA     BIT       PWM0S
      000000F0H.7 SFRSYM    DATA     BIT       B7
      000000E0H.1 SFRSYM    DATA     BIT       ACC1
      000000F8H.4 SFRSYM    DATA     BIT       XCLKF
      000000E0H.2 SFRSYM    DATA     BIT       ACC2
      0000008EH   SFRSYM    DATA     BYTE      PDSEL
      000000E0H.3 SFRSYM    DATA     BIT       ACC3
      000000D0H   SFRSYM    DATA     BYTE      PSW
      000000E0H.4 SFRSYM    DATA     BIT       ACC4
      00000098H.2 SFRSYM    DATA     BIT       RB80
      000000E0H.5 SFRSYM    DATA     BIT       ACC5
      000000FDH   SFRSYM    DATA     BYTE      ADCVREF
      000000E0H.6 SFRSYM    DATA     BIT       ACC6

      01000A70H   BLOCK     CODE     ---       LVL=0
      01000A70H   LINE      CODE     ---       #13
      01000A70H   LINE      CODE     ---       #14
      01000A70H   LINE      CODE     ---       #15
      01000A73H   LINE      CODE     ---       #17
LX51 LINKER/LOCATER V4.66.97.0                                                        07/19/2022  10:30:28  PAGE 32


      01000A76H   LINE      CODE     ---       #19
      01000A79H   LINE      CODE     ---       #21
      01000A79H   LINE      CODE     ---       #22
      01000A79H   LINE      CODE     ---       #24
      ---         BLOCKEND  ---      ---       LVL=0

      ---         MODULE    ---      ---       ?C_INIT
      01000885H   PUBLIC    CODE     ---       ?C_START

      ---         MODULE    ---      ---       ?C?CLDPTR
      010003C3H   PUBLIC    CODE     ---       ?C?CLDPTR

      ---         MODULE    ---      ---       ?C?CLDOPTR
      010003DCH   PUBLIC    CODE     ---       ?C?CLDOPTR

      ---         MODULE    ---      ---       ?C?ILDIX
      01000409H   PUBLIC    CODE     ---       ?C?ILDIX

      ---         MODULE    ---      ---       ?C?LADD
      0100041FH   PUBLIC    CODE     ---       ?C?LADD

      ---         MODULE    ---      ---       ?C?LMUL
      0100042CH   PUBLIC    CODE     ---       ?C?LMUL

      ---         MODULE    ---      ---       ?C?ULDIV
      010004B7H   PUBLIC    CODE     ---       ?C?ULDIV

      ---         MODULE    ---      ---       ?C?LOR
      01000549H   PUBLIC    CODE     ---       ?C?LOR

      ---         MODULE    ---      ---       ?C?ULCMP
      01000556H   PUBLIC    CODE     ---       ?C?ULCMP

      ---         MODULE    ---      ---       ?C?ULSHR
      01000567H   PUBLIC    CODE     ---       ?C?ULSHR

      ---         MODULE    ---      ---       ?C?LSHL
      0100057AH   PUBLIC    CODE     ---       ?C?LSHL

      ---         MODULE    ---      ---       ?C?LLDOPTR
      0100058DH   PUBLIC    CODE     ---       ?C?LLDOPTR

      ---         MODULE    ---      ---       ?C?LLDXDATA
      010005BDH   PUBLIC    CODE     ---       ?C?LLDXDATA

      ---         MODULE    ---      ---       ?C?LLDXDATA0
      010005C9H   PUBLIC    CODE     ---       ?C?LLDXDATA0

      ---         MODULE    ---      ---       ?C?LLDIXDATA
      010005DEH   PUBLIC    CODE     ---       ?C?LLDIXDATA
      010005D5H   PUBLIC    CODE     ---       ?C?LLDIXDATA1
      010005D7H   PUBLIC    CODE     ---       ?C?LLDIXDATA8

      ---         MODULE    ---      ---       ?C?LSTXDATA
      0100060AH   PUBLIC    CODE     ---       ?C?LSTXDATA

      ---         MODULE    ---      ---       ?C?LSTKXDATA
      01000616H   PUBLIC    CODE     ---       ?C?LSTKXDATA

      ---         MODULE    ---      ---       ?C?PLDXDATA
      01000647H   PUBLIC    CODE     ---       ?C?PLDXDATA

      ---         MODULE    ---      ---       ?C?PLDIXDATA
      01000650H   PUBLIC    CODE     ---       ?C?PLDIXDATA

LX51 LINKER/LOCATER V4.66.97.0                                                        07/19/2022  10:30:28  PAGE 33


      ---         MODULE    ---      ---       ?C?PSTXDATA
      01000667H   PUBLIC    CODE     ---       ?C?PSTXDATA

      ---         MODULE    ---      ---       ?C?LCASE
      01000670H   PUBLIC    CODE     ---       ?C?LCASE

      ---         MODULE    ---      ---       ?C?ICALL
      010006AAH   PUBLIC    CODE     ---       ?C?ICALL
      010006AEH   PUBLIC    CODE     ---       ?C?ICALL2

      ---         MODULE    ---      ---       PRINTF
      02000045H   PUBLIC    XDATA    ---       ?_PRINTF517?BYTE
      02000045H   PUBLIC    XDATA    ---       ?_PRINTF?BYTE
      02000045H   PUBLIC    XDATA    ---       ?_SPRINTF517?BYTE
      02000045H   PUBLIC    XDATA    ---       ?_SPRINTF?BYTE
      010000C9H   PUBLIC    CODE     ---       _PRINTF
      010000C9H   PUBLIC    CODE     ---       _PRINTF517
      010000C3H   PUBLIC    CODE     ---       _SPRINTF
      010000C3H   PUBLIC    CODE     ---       _SPRINTF517

      ---         MODULE    ---      ---       ?C?CSTPTR
      010006B0H   PUBLIC    CODE     ---       ?C?CSTPTR

      ---         MODULE    ---      ---       ?C?LLDIDATA
      010006C2H   PUBLIC    CODE     ---       ?C?LLDIDATA

      ---         MODULE    ---      ---       ?C?LLDPDATA
      010006CEH   PUBLIC    CODE     ---       ?C?LLDPDATA

      ---         MODULE    ---      ---       ?C?LLDCODE
      010006DAH   PUBLIC    CODE     ---       ?C?LLDCODE

      ---         MODULE    ---      ---       ?C?CCASE
      010006EAH   PUBLIC    CODE     ---       ?C?CCASE

Program Size: data=15.1 xdata=122 const=51 code=2686
LX51 RUN COMPLETE.  0 WARNING(S),  0 ERROR(S)
